:0300000002684A49
:10684A00758E1190000078FF79FFE4F0A3D9FBD888
:0D685A00F778FFE4F6D8FD75817F0268A293
:106C3D004401EA40490FDB4401E640C90FDB440142
:056C4D00E23C8EFA3567
:06494E009001CA122011C5
:104954009001CEE0FCA3E0FDA3E0FEA3E0FFEF2482
:1049640069FFEE3474FEED34FFFDEC34FFFCEC1211
:104974001B7B7BDF7A927986783D1219579001D29E
:104984001220117B007A0079C078419001D2E0FCBA
:10499400A3E0FDA3E0FEA3E0FF121A601260B67B61
:1049A400007A0079C07841121957C004C005C006C6
:1049B400C0077F977E7E7DD57C409001D2E0F8A32E
:1049C400E0F9A3E0FAA3E0FB121866D003D002D00A
:1049D40001D000121862C004C005C006C0077F924F
:1049E4007E867DC07C419001CAE0F8A3E0F9A3E093
:1049F400FAA3E0FB121957A804A905AA06AB07D02D
:104A040007D006D005D0041218669001DA122011DE
:104A14009001CEE0FCA3E0FDA3E0FEA3E0FFEF24C1
:104A240069FFEE3474FEED34FFFDEC34FFFCEC1250
:104A34001B7B9001CAE0F8A3E0F9A3E0FAA3E0FB32
:104A44001218667B307AE67958783D121957A80413
:104A5400A905AA06AB077F817E0E7DBA7C43121896
:104A6400629001E2E0F8A3E0F9A3E0FAA3E0FB120C
:104A740019579001D61220119001E6E0FCA3E0FD45
:104A8400A3E0FEA3E0FF9001D6E0F8A3E0F9A3E0E1
:104A9400FAA3E0FB121AFD602940279001D6E0FC3E
:104AA400A3E0FDA3E0FEA3E0FF9001E6E0F8A3E0AD
:104AB400F9A3E0FAA3E0FB1218629001D6122011C8
:104AC40080B69001E6E0FCA3E0FDA3E0FEA3E0FFD6
:104AD400121B6A9001D6E0F8A3E0F9A3E0FAA3E080
:104AE400FB121AFD50279001D6E0FCA3E0FDA3E0E1
:104AF400FEA3E0FF9001E6E0F8A3E0F9A3E0FAA347
:104B0400E0FB1218669001D612201180B57F007E5A
:104B1400007D007C009001D6E0F8A3E0F9A3E0FA60
:104B2400A3E0FB121AFD604840469001EAE0FCA3B2
:104B3400E0FDA3E0FEA3E0FF9001D6E0F8A3E0F9D6
:104B4400A3E0FAA3E0FB121AFD50259001D6E0FC85
:104B5400A3E0FDA3E0FEA3E0FF9001E6E0F8A3E0FC
:104B6400F9A3E0FAA3E0FB1218629001D612201117
:104B74007F007E007D007C009001D6E0F8A3E0F980
:104B8400A3E0FAA3E0FB121AFD504B9001EAE0FC0B
:104B9400A3E0FDA3E0FEA3E0FF121B6A9001D6E0B0
:104BA400F8A3E0F9A3E0FAA3E0FB121AFD602740A2
:104BB400259001D6E0FCA3E0FDA3E0FEA3E0FF9076
:104BC40001E6E0F8A3E0F9A3E0FAA3E0FB1218661B
:104BD4009001D61220119001D6E0FCA3E0FDA3E0E1
:104BE400FEA3E0FF12591C7B247A0B7998783912C2
:104BF40019579001DAE0F8A3E0F9A3E0FAA3E0FB87
:104C04001218669001DE1220117B007A0079C078B8
:104C1400419001DEE0FCA3E0FDA3E0FEA3E0FF126F
:104C24001A601260B67B007A0079C0784112195775
:104C3400A804A905AA06AB079001DEE0FCA3E0FDE9
:094C4400A3E0FEA3E0FF121862D8
:014C4D002244
:106CCA009001F51220119001F5E0FCA3E0FDA3E08C
:106CDA00FEA3E0FF1260B6A804A905AA06AB0790B6
:106CEA0001F5E0FCA3E0FDA3E0FEA3E0FF121862B9
:106CFA009001E6E0F8A3E0F9A3E0FAA3E0FB121999
:026D0A0057220E
:060D300090015A1220118F
:100D360090015AE0FCA3E0FDA3E0FEA3E0FFEF2450
:100D460013FFEE342DFEED34FFFDEC34FFFCEC1208
:100D56001B7B90015EE0F8A3E0F9A3E0FAA3E0FBB9
:100D66001218669001621220117F8D7EA67D147C7A
:100D76003D900162E0F8A3E0F9A3E0FAA3E0FB12DC
:100D860019577B807AF279BF783E121866126CCAC0
:100D96009001661220117F477E857D167C3D90016D
:100DA60062E0F8A3E0F9A3E0FAA3E0FB1219577B8F
:100DB600937AA77984783E121866126CCA90016AF3
:100DC6001220117F217EB47D0A7C3D900162E0F8FD
:100DD600A3E0F9A3E0FAA3E0FB1219577BFF7ACD53
:100DE6007953783F121866126CCA90016E12201160
:100DF6007F4D7E6C7D337C3B900162E0F8A3E0F989
:100E0600A3E0FAA3E0FB1219577B817A3D797E783D
:100E16003F121866126CCA9001721220117F007E72
:100E2600007D007C4090016EE0F8A3E0F9A3E0FAB3
:100E3600A3E0FB121957A804A905AA06AB0790015F
:100E460066E0FCA3E0FDA3E0FEA3E0FF1218621239
:100E560059067BF37A767914783F121957C004C085
:100E660005C006C007900166E0FCA3E0FDA3E0FE16
:100E7600A3E0FF1259067BE87AC17951784012192E
:100E860057A804A905AA06AB077FB17E737D717CBE
:100E960042121862D003D002D001D000121862C0EC
:100EA60004C005C006C0077F007E007D007C409020
:100EB600016EE0F8A3E0F9A3E0FAA3E0FB121957EC
:100EC6001259067B0C7A5979ED783E121957A80407
:100ED600A905AA06AB07D007D006D005D00412187C
:100EE600629001761220117F007E007D007C40908A
:100EF600016EE0F8A3E0F9A3E0FAA3E0FB121957AC
:100F0600C004C005C006C0077F007E007D007C408F
:100F1600900166E0F8A3E0F9A3E0FAA3E0FB12195A
:100F260057D003D002D001D0001218621259067BA6
:100F3600767A4F791E783D121957C004C005C0064F
:100F4600C0077F007E007D007C40900166E0F8A32C
:100F5600E0F9A3E0FAA3E0FB1219571259067B9CAD
:100F66007A5A79B6783D121957A804A905AA06AB8C
:100F760007900176E0FCA3E0FDA3E0FEA3E0FF12EC
:100F86001862A804A905AA06AB07D007D006D005A3
:100F9600D004121866C004C005C006C0077F007ED4
:100FA600007D007C4090016EE0F8A3E0F9A3E0FA32
:100FB600A3E0FB121957900172E0F8A3E0F9A3E051
:100FC600FAA3E0FB1218621259067B687A96790436
:100FD600783D121957A804A905AA06AB07D007D071
:100FE60006D005D0041218629001761220117F00F7
:100FF6007E007D007C4090016EE0F8A3E0F9A3E05E
:10100600FAA3E0FB121957A804A905AA06AB079094
:101016000166E0FCA3E0FDA3E0FEA3E0FF12186278
:10102600900172E0F8A3E0F9A3E0FAA3E0FB12183E
:10103600661259067BD87A2A79C1783C121957C0AC
:1010460004C005C006C0077F007E007D007C40907E
:10105600016EE0F8A3E0F9A3E0FAA3E0FB1219574A
:10106600A804A905AA06AB07900166E0FCA3E0FD6B
:10107600A3E0FEA3E0FF1218621259067B727A33D0
:1010860079DC783C121957A804A905AA06AB079083
:101096000176E0FCA3E0FDA3E0FEA3E0FF121862E8
:1010A600D003D002D001D000121862C004C005C01F
:1010B60006C007900172E0F8A3E0F9A3E0FAA3E006
:1010C600FB900166E0FCA3E0FDA3E0FEA3E0FF12B7
:1010D60018621259067B307A4C79A6783C12195759
:1010E600A804A905AA06AB07D007D006D005D004E8
:1010F60012186290017612201190016EE0FCA3E0B6
:10110600FDA3E0FEA3E0FF1259067B0B7AD2798C91
:10111600783C121957900176E0F8A3E0F9A3E0FABB
:10112600A3E0FB121866C004C005C006C007900104
:1011360072E0FCA3E0FDA3E0FEA3E0FF900166E001
:10114600F8A3E0F9A3E0FAA3E0FB12186612590629
:101156007B697AE37988783C121957A804A905AA0D
:1011660006AB07D007D006D005D00412186690014A
:10117600761220117F007E007D007C4090016AE09F
:10118600F8A3E0F9A3E0FAA3E0FB121957A804A913
:1011960005AA06AB07900166E0FCA3E0FDA3E0FE0E
:1011A600A3E0FF1218621259067BF97A4E794C7841
:1011B6003C121957C004C005C006C007900172E072
:1011C600FCA3E0FDA3E0FEA3E0FF1259067BCD7A67
:1011D600AF79E6783B121957A804A905AA06AB070A
:1011E600D007D006D005D004121866C004C005C0CA
:1011F60006C0077F007E007D007C4090016EE0F80F
:10120600A3E0F9A3E0FAA3E0FB121957900172E0FC
:10121600F8A3E0F9A3E0FAA3E0FB12186612590658
:101226007BBC7A5779AD783B121957A804A905AA51
:1012360006AB07D007D006D005D004121866C00446
:10124600C005C006C0077F007E007D807C409001FF
:101256006EE0F8A3E0F9A3E0FAA3E0FB121957A8A1
:1012660004A905AA06AB07900166E0FCA3E0FDA36E
:10127600E0FEA3E0FF1218621259067B4E7AB4799B
:10128600AB783B121957A804A905AA06AB07D007E5
:10129600D006D005D00412186290017A1220117F70
:1012A600007E007D007C4090016EE0F8A3E0F9A38B
:1012B600E0FAA3E0FB121957A804A905AA06AB0792
:1012C600900166E0FCA3E0FDA3E0FEA3E0FF121898
:1012D60062900172E0F8A3E0F9A3E0FAA3E0FB1242
:1012E60018621259067BA97A6A7982783B121957D5
:1012F60090017AE0F8A3E0F9A3E0FAA3E0FB121864
:1013060066C004C005C006C0077F007E007D407C25
:1013160040900166E0F8A3E0F9A3E0FAA3E0FB122F
:1013260019571259067B9C7ADC796F783B1219574C
:10133600A804A905AA06AB07D007D006D005D00495
:10134600121862C004C005C006C0077F007E007D7B
:10135600807C4090016EE0F8A3E0F9A3E0FAA3E0F8
:10136600FB121957C004C005C006C0077F007E00E7
:101376007D007C40900166E0F8A3E0F9A3E0FAA3C3
:10138600E0FB121957D003D002D001D00012186228
:101396001259067BCA7A547941783B121957A80428
:1013A600A905AA06AB07D007D006D005D0041218A7
:1013B6006290017A1220117F007E007D007C4090B1
:1013C600016EE0F8A3E0F9A3E0FAA3E0FB121957D7
:1013D600C004C005C006C0077F007E007D407C407B
:1013E600900166E0F8A3E0F9A3E0FAA3E0FB121986
:1013F60057D003D002D001D0001218621259067BD2
:10140600457A2F7923783B121957C004C005C006C8
:10141600C007900172E0FCA3E0FDA3E0FEA3E0FF9D
:1014260090016EE0F8A3E0F9A3E0FAA3E0FB12183E
:10143600661259067B147A5C792C783B121957A8E8
:1014460004A905AA06AB0790017AE0FCA3E0FDA378
:10145600E0FEA3E0FF121862A804A905AA06AB07DE
:10146600D007D006D005D004121866C004C005C047
:1014760006C0077F007E007D007C4090016EE0F88C
:10148600A3E0F9A3E0FAA3E0FB121957900166E086
:10149600F8A3E0F9A3E0FAA3E0FB12186690017244
:1014A600E0F8A3E0F9A3E0FAA3E0FB1218621259F0
:1014B600067BA67AD57910783B121957A804A90598
:1014C600AA06AB07D007D006D005D004121862C012
:1014D60004C005C006C0077F007E007D007C4090EA
:1014E600016EE0F8A3E0F9A3E0FAA3E0FB121957B6
:1014F600C004C005C006C0077F007E007D007C409A
:1015060090016AE0F8A3E0F9A3E0FAA3E0FB121960
:1015160057D003D002D001D0001218621259067BB0
:10152600B37A7B79F2783A121957A804A905AA0664
:10153600AB07D007D006D005D00412186690017A02
:101546001220117F007E007D007C4090016AE0F849
:10155600A3E0F9A3E0FAA3E0FB121957900166E0B5
:10156600F8A3E0F9A3E0FAA3E0FB121866C004C0F2
:1015760005C006C0077F007E007D007C4090016E9E
:10158600E0F8A3E0F9A3E0FAA3E0FB121957A804D8
:10159600A905AA06AB07D007D006D005D0041218B5
:1015A600621259067B047AAD79C0783A121957C08F
:1015B60004C005C006C0077F007E007D007C409009
:1015C6000172E0F8A3E0F9A3E0FAA3E0FB121957D1
:1015D600C004C005C006C0077F007E007D007C40B9
:1015E60090016EE0F8A3E0F9A3E0FAA3E0FB12197C
:1015F60057D003D002D001D0001218621259067BD0
:10160600A37A0679D378BA121957A804A905AA06A7
:10161600AB07D007D006D005D004121866C004C0A8
:1016260005C006C0077F007E007D807C4090016E6D
:10163600E0F8A3E0F9A3E0FAA3E0FB121957125968
:10164600067B4B7A1F79BA783A121957A804A9056E
:10165600AA06AB07D007D006D005D004121862C080
:1016660004C005C006C0077F007E007D007C409058
:10167600016EE0F8A3E0F9A3E0FAA3E0FB12195724
:10168600C004C005C006C0077F007E007D007C4008
:10169600900166E0F8A3E0F9A3E0FAA3E0FB1219D3
:1016A60057D003D002D001D000121862900172E028
:1016B600F8A3E0F9A3E0FAA3E0FB121866125906B4
:1016C6007BA97A3079B6783A121957A804A905AADF
:1016D60006AB07D007D006D005D0041218669001D5
:1016E6007E1220117F007E007D807C4090016EE09E
:1016F600F8A3E0F9A3E0FAA3E0FB121957A804A99E
:1017060005AA06AB07900166E0FCA3E0FDA3E0FE98
:10171600A3E0FF121862900172E0F8A3E0F9A3E0DB
:10172600FAA3E0FB1218661259067B3B7AAA799A4D
:10173600783A121957A804A905AA06AB0790017EA4
:10174600E0FCA3E0FDA3E0FEA3E0FF121862C004E4
:10175600C005C006C0077F007E007D007C4090016A
:101766006EE0F8A3E0F9A3E0FAA3E0FB121957C074
:1017760004C005C006C0077F007E007D007C409047
:101786000166E0F8A3E0F9A3E0FAA3E0FB1219571B
:10179600A804A905AA06AB07D007D006D005D00431
:1017A6001218661259067B247A0B7998783A121920
:1017B60057A804A905AA06AB07D007D006D005D0BE
:1017C60004121862C004C005C006C0077F007E0070
:1017D6007D007C40900166E0F8A3E0F9A3E0FAA35F
:1017E600E0FB121957900172E0F8A3E0F9A3E0FAC2
:1017F600A3E0FB1218621259067BE07A2D799078E5
:101806003A121957A804A905AA06AB07D007D006AD
:10181600D005D00412186290017E12201190017A30
:10182600E0FCA3E0FDA3E0FEA3E0FF900176E0F874
:10183600A3E0F9A3E0FAA3E0FB12186690017EE0AC
:10184600F8A3E0F9A3E0FAA3E0FB1218667B487A56
:081856005179C77845121957BA
:01185E002267
:0B2AB600900120EBF0A3EAF0A3E9F090
:102AC100900126E0FCA3E0FDA3E0FEA3E0FFEC12F1
:102AD1001B7B7B007A81798878C612186690012A5F
:102AE100E0F8A3E0F9A3E0FAA3E0FB121866900175
:102AF1002E1220117F0A7EEB7D157C3D90012EE088
:102B0100F8A3E0F9A3E0FAA3E0FB1219577B7F7A5F
:102B11004F7940783F121866126CCA900132122028
:102B2100117F8C7EA67D147C3D90012EE0F8A3E000
:102B3100F9A3E0FAA3E0FB1219577B367A90795298
:102B4100783F121866126CCA9001361220117F4D1F
:102B51007E6C7D337C3B90012EE0F8A3E0F9A3E08D
:102B6100FAA3E0FB1219577B857AEA797E783F1246
:102B71001866126CCA90013A1220117F217EB47D31
:102B81000A7C3D90012EE0F8A3E0F9A3E0FAA3E06E
:102B9100FB1219577BD37A697979783F121866123B
:102BA1006CCA90013E1220117F477E857D167C3DC7
:102BB10090012EE0F8A3E0F9A3E0FAA3E0FB1219DB
:102BC100577B9F7A027900783D121866126CCA9081
:102BD10001421220117F007E007D007C4090013E69
:102BE100E0F8A3E0F9A3E0FAA3E0FB1219571259A8
:102BF1001C7BB07A727928783F121957C004C0053E
:102C0100C006C007900136E0FCA3E0FDA3E0FEA3EF
:102C1100E0FF12591C7B7D7A3F79C9784012195720
:102C2100A804A905AA06AB07D007D006D005D00491
:102C3100121866C004C005C006C0077F007E007D73
:102C4100007C4090013EE0F8A3E0F9A3E0FAA3E0A4
:102C5100FB121957A804A905AA06AB07900136E093
:102C6100FCA3E0FDA3E0FEA3E0FF12186212591CD1
:102C71007B6F7A1279A3783F121957A804A905AA84
:102C810006AB07D007D006D005D004121862C004E5
:102C9100C005C006C00790013AE0FCA3E0FDA3E037
:102CA100FEA3E0FF12591C7BC97A76793E783E1269
:102CB1001957A804A905AA06AB07D007D006D00565
:102CC100D0041218629001E2E0F8A3E0F9A3E0FA5F
:102CD100A3E0FB121957900132E0F8A3E0F9A3E059
:102CE100FAA3E0FB121866900146122011900146EA
:102CF100E0FCA3E0FDA3E0FEA3E0FFC004C005C02B
:102D010006C0077F007E007D007C40900142E0F814
:102D1100A3E0F9A3E0FAA3E0FB12195712591C7BB7
:102D2100D57A7879E9783D121957C004C005C006F3
:102D3100C0077F007E007D007C40900136E0F8A353
:102D4100E0F9A3E0FAA3E0FB12195712591C7BD159
:102D51007A22795B783E121957D003D002D001D084
:102D610000121862C004C005C006C0077F007E00C3
:102D71007D007C4090013EE0F8A3E0F9A3E0FAA3D6
:102D8100E0FB121957C004C005C006C0077F007ED2
:102D9100007D007C40900136E0F8A3E0F9A3E0FA61
:102DA100A3E0FB121957D003D002D001D0001218B2
:102DB1006212591C7BFC7AA97971783D121957A8C6
:102DC10004A905AA06AB07D007D006D005D0041286
:102DD1001862C004C005C006C0077F007E007D00E8
:102DE1007C4090013EE0F8A3E0F9A3E0FAA3E0FB08
:102DF100121957C004C005C006C00790013AE0FC93
:102E0100A3E0FDA3E0FEA3E0FF900136E0F8A3E01C
:102E1100F9A3E0FAA3E0FB121866D003D002D001B7
:102E2100D00012186212591C7BD57A787969783DE5
:102E3100121957A804A905AA06AB07D007D006D0D6
:102E410005D0041218629001E2E0F8A3E0F9A3E0D2
:102E5100FAA3E0FB121957A804A905AA06AB07D0EB
:102E610007D006D005D00412186690014612201131
:102E71007F007E007D007C4090013EE0F8A3E0F9F8
:102E8100A3E0FAA3E0FB12195712591C7BE37AC79E
:102E91007928783F121957C004C005C006C00790B1
:102EA1000136E0FCA3E0FDA3E0FEA3E0FF12591C04
:102EB1007B9E7A5E79C77840121957A804A905AAA2
:102EC10006AB07D007D006D005D004121866C0049F
:102ED100C005C006C0077F007E007D007C409001D8
:102EE1003EE0F8A3E0F9A3E0FAA3E0FB121957A82A
:102EF10004A905AA06AB07900136E0FCA3E0FDA3F7
:102F0100E0FEA3E0FF12186212591C7BE57AD0792A
:102F1100A2783F121957A804A905AA06AB07D00742
:102F2100D006D005D0041218629001E2E0F8A3E0C7
:102F3100F9A3E0FAA3E0FB121957900142E0F8A3CC
:102F4100E0F9A3E0FAA3E0FB12186690014A12200F
:102F5100117F007E007D007C4090013EE0F8A3E0FF
:102F6100F9A3E0FAA3E0FB121957A804A905AA06E0
:102F7100AB07900142E0FCA3E0FDA3E0FEA3E0FF6C
:102F810012186212591C7B067A817915783E121942
:102F910057C004C005C006C00790014AE0FCA3E089
:102FA100FDA3E0FEA3E0FF12591C7BA67A9B79A446
:102FB1007840121957D003D002D001D00012186204
:102FC1009001E2E0F8A3E0F9A3E0FAA3E0FB121913
:102FD1005790014E122011900146E0FCA3E0FDA3A1
:102FE100E0FEA3E0FF12591CC004C005C006C007E3
:102FF10090014EE0FCA3E0FDA3E0FEA3E0FF125927
:1030010006A804A905AA06AB07D007D006D005D0AB
:10301100041219577B327AAF79CB783E121957C017
:1030210004C005C006C00790014EE0FCA3E0FDA36B
:10303100E0FEA3E0FF12591C7BDB7ADE796A783F60
:10304100121957A804A905AA06AB07D007D006D0C4
:1030510005D004121866900123E0FBA3E0FAA3E077
:10306100F9121F9F900123E0FBA3E0FAA3E0F912FC
:103071001F7F900123E0FBA3E0FAA3E0F9121FF107
:10308100121957A804A905AA06AB077F007E007D87
:10309100807C3F12186212665B9000E8122011904A
:1030A1000123E0FBA3E0FAA3E0F9121F7F1268E716
:1030B100900123E0FBA3E0FAA3E0F9121F9F900126
:1030C10046E0FCA3E0FDA3E0FEA3E0FF125906C029
:1030D10004C005C006C00790014EE0FCA3E0FDA3BB
:1030E100E0FEA3E0FF125906A804A905AA06AB0752
:1030F100D007D006D005D004121957C004C005C0AE
:1031010006C007900123E0FBA3E0FAA3E0F9121F38
:103111007F125906A804A905AA06AB07D007D00655
:10312100D005D004121A609001521220119001466C
:10313100E0FCA3E0FDA3E0FEA3E0FF12591CC004E4
:10314100C005C006C00790014EE0FCA3E0FDA3E06E
:10315100FEA3E0FF125906A804A905AA06AB07D0F1
:1031610007D006D005D0041219577BDB7ADE796AC5
:10317100783F121957C004C005C006C00790014E20
:10318100E0FCA3E0FDA3E0FEA3E0FF12591C7B32AB
:103191007AAF79CB783E121957A804A905AA06ABD4
:1031A10007D007D006D005D004121862C004C005AC
:1031B100C006C007900123E0FBA3E0FAA3E0F912E7
:1031C1001F7F125906A804A905AA06AB07D007D08C
:1031D10006D005D004121A609001561220119001F8
:1031E10056E0FCA3E0FDA3E0FEA3E0FFC004C005A0
:1031F100C006C007900152E0FCA3E0FDA3E0FEA3DE
:10320100E0FF9000E8122011D007D006D005D004CD
:103211001268E7900120E0FBA3E0FAA3E0F9121F96
:103221009F900120E0FBA3E0FAA3E0F9121F7F7B4E
:10323100007A0079007800121AFD6030402E90016A
:1032410020E0FBA3E0FAA3E0F9C003C002C0011231
:103251001F7F9001E6E0F8A3E0F9A3E0FAA3E0FB09
:10326100121866D001D002D003121F9F900120E0F6
:10327100FBA3E0FAA3E0F9121F7F9001E6E0F8A3B7
:10328100E0F9A3E0FAA3E0FB121AFD502E90012011
:10329100E0FBA3E0FAA3E0F9C003C002C001121FE2
:1032A1007F9001E6E0F8A3E0F9A3E0FAA3E0FB12C6
:0B32B1001862D001D002D003121F9F52
:0132BC0022EF
:0B4586009001A8EBF0A3EAF0A3E9F01D
:104591009001AEE0FCA3E0FDA3E0FEA3E0FFEC127E
:1045A1001B7B7B007A81798878C61218669001B2EC
:1045B100E0F8A3E0F9A3E0FAA3E0FB1218667B00A0
:1045C1007AAD790E7847121A609001B61220117FE8
:1045D100A67EFE7DC77C429001B6E0F8A3E0F9A378
:1045E100E0FAA3E0FB1219577B917AEA797E783FD2
:1045F100121866126CCA9001BA1220117F117E2323
:104601007D5F7C379001B6E0F8A3E0F9A3E0FAA35F
:10461100E0FB121957A804A905AA06AB077F507E33
:10462100AC7DAE7C3B121862126CCAC004C005C0DE
:1046310006C0079001BAE0FCA3E0FDA3E0FEA3E001
:10464100FF12591CA804A905AA06AB07D007D0067A
:10465100D005D004121957C004C005C006C0077F99
:10466100187E017DC87C429001B6E0F8A3E0F9A371
:10467100E0FAA3E0FB1219577B327AE47946783FDE
:10468100121866126CCAA804A905AA06AB07D007BE
:10469100D006D005D004121866C004C005C006C0FB
:1046A100077F007E007D007C409001BAE0F8A3E026
:1046B100F9A3E0FAA3E0FB12195712591C7B0C7AFB
:1046C1003479697838121957A804A905AA06AB07E5
:1046D100D007D006D005D0041218669001BE122072
:1046E100117F147E6A7D177C389001B6E0F8A3E053
:1046F100F9A3E0FAA3E0FB121957A804A905AA0639
:10470100AB077F6D7E6A7D857C3D121862126CCA93
:104711009001C21220119001BEE0FCA3E0FDA3E0D4
:10472100FEA3E0FF125958C004C005C006C007909F
:1047310001C2E0FCA3E0FDA3E0FEA3E0FF125906E5
:10474100A804A905AA06AB07D007D006D005D00456
:10475100121957125A669001A8E0FBA3E0FAA3E0F0
:10476100F9121F9F9001E6E0F8A3E0F9A3E0FAA394
:10477100E0FB9001BEE0FCA3E0FDA3E0FEA3E0FFAF
:10478100121A601260B69001E6E0F8A3E0F9A3E026
:10479100FAA3E0FB121957A804A905AA06AB0790D2
:1047A10001BEE0FCA3E0FDA3E0FEA3E0FF1218625E
:1047B1009001C61220117F007E007DC07C3F9001D8
:1047C100EAE0F8A3E0F9A3E0FAA3E0FB121957909D
:1047D10001C6E0F8A3E0F9A3E0FAA3E0FB121AFD99
:1047E100505A7F007E007D007C3F9001EAE0F8A3F3
:1047F100E0F9A3E0FAA3E0FB1219579001C6E0F833
:10480100A3E0F9A3E0FAA3E0FB121AFD402E900108
:10481100A8E0FBA3E0FAA3E0F9C003C002C00112C3
:104821001F7F9001EAE0F8A3E0F9A3E0FAA3E0FB1F
:10483100121866D001D002D003121F9F9001A8E088
:10484100FBA3E0FAA3E0F9C003C002C001121F7F7D
:10485100C004C005C006C0079001A8E0FBA3E0FAB0
:10486100A3E0F9121F7F9001E6E0F8A3E0F9A3E0CD
:10487100FAA3E0FB121A601260B69001E6E0F8A319
:10488100E0F9A3E0FAA3E0FB121957A804A905AACD
:1048910006AB07D007D006D005D004121862D001AC
:1048A100D002D003121F9F9001BEE0FCA3E0FDA344
:1048B100E0FEA3E0FF12591CC004C005C006C007FA
:1048C1009001C2E0FCA3E0FDA3E0FEA3E0FF1259CA
:1048D1001CA804A905AA06AB07D007D006D005D0AD
:1048E100041219579001ABE0FBA3E0FAA3E0F9121F
:1048F1001F9F9001ABE0FBA3E0FAA3E0F9121F7F39
:104901009001ABE0FBA3E0FAA3E0F9121FF1121949
:1049110057A804A905AA06AB077F007E007D807C0D
:104921003F12186212665B9000E81220119001ABF1
:10493100E0FBA3E0FAA3E0F9121F7F1268E7900100
:0C494100ABE0FBA3E0FAA3E0F9121F9F1B
:01494D002247
:0B32BD00900182EBF0A3EAF0A3E9F01F
:1032C8007F927E0A7D867C3E900188E0F8A3E0F933
:1032D800A3E0FAA3E0FB12195790018CE0F8A3E0F1
:1032E800F9A3E0FAA3E0FB121862900194122011EE
:1032F8007F007E007D007C00900194E0F8A3E0F957
:10330800A3E0FAA3E0FB121AFD5027900194E0FC19
:10331800A3E0FDA3E0FEA3E0FF9001E6E0F8A3E050
:10332800F9A3E0FAA3E0FB121866900194122011A9
:1033380080489001E6E0FCA3E0FDA3E0FEA3E0FFE7
:10334800900194E0F8A3E0F9A3E0FAA3E0FB121AD5
:10335800FD60274025900194E0FCA3E0FDA3E0FE7A
:10336800A3E0FF9001E6E0F8A3E0F9A3E0FAA3E008
:10337800FB121862900194122011900194E0F8A3B6
:10338800E0F9A3E0FAA3E0FB90001EE0FCA3E0FD57
:10339800A3E0FEA3E0FF121862900016122011901D
:1033A8000016E0FCA3E0FDA3E0FEA3E0FF1259062F
:1033B800C004C005C006C00790001AE0FCA3E0FDE9
:1033C800A3E0FEA3E0FF125906A804A905AA06ABCC
:1033D80007D007D006D005D004121957C004C0057D
:1033E800C006C007900190E0FCA3E0FDA3E0FEA3A7
:1033F800E0FF125906A804A905AA06AB07D007D012
:1034080006D005D004121957C004C005C006C0076D
:1034180090001AE0FCA3E0FDA3E0FEA3E0FF125930
:103428001CC004C005C006C007900190E0FCA3E0E2
:10343800FDA3E0FEA3E0FF12591CA804A905AA06F3
:10344800AB07D007D006D005D004121957A804A995
:1034580005AA06AB07D007D006D005D00412186617
:10346800900198122011900198E0FCA3E0FDA3E0E0
:10347800FEA3E0FF900198E0F8A3E0F9A3E0FAA327
:10348800E0FB121957A804A905AA06AB077F007E1E
:10349800007D807C3F12186212665B90019C1220AE
:1034A80011900198E0FCA3E0FDA3E0FEA3E0FFC0BB
:1034B80004C005C006C00790019CE0FCA3E0FDA382
:1034C800E0FEA3E0FF9000E8122011D007D006D05C
:1034D80005D0041268E7900185E0FBA3E0FAA3E0B9
:1034E800F9121F9F900185E0FBA3E0FAA3E0F9120F
:1034F8001F7F125906C004C005C006C00790018589
:10350800E0FBA3E0FAA3E0F9121F7F12591CD003D5
:10351800D002D001D000121A60C004C005C006C095
:103528000790001AE0FCA3E0FDA3E0FEA3E0FF1271
:103538005906C004C005C006C00790001AE0FCA3E5
:10354800E0FDA3E0FEA3E0FF12591CD003D002D097
:1035580001D000121A60A804A905AA06AB07D00773
:10356800D006D005D004121957C004C005C006C043
:1035780007900185E0FBA3E0FAA3E0F9121F7F1290
:103588005906C004C005C006C00790001AE0FCA395
:10359800E0FDA3E0FEA3E0FF125906A804A905AACE
:1035A80006AB07D007D006D005D004121957C004BF
:1035B800C005C006C007900190E0FCA3E0FDA3E0B1
:1035C800FEA3E0FF12591CD003D002D001D0001294
:1035D8001A60D003D002D001D0001218629001A462
:1035E800122011900190E0FCA3E0FDA3E0FEA3E00F
:1035F800FF125906C004C005C006C00790001AE0B3
:10360800FCA3E0FDA3E0FEA3E0FF125906A804A96D
:1036180005AA06AB07D007D006D005D00412195763
:10362800C004C005C006C007900016E0FCA3E0FD7A
:10363800A3E0FEA3E0FF125906A804A905AA06AB59
:1036480007D007D006D005D004121957C004C0050A
:10365800C006C007900190E0FCA3E0FDA3E0FEA334
:10366800E0FF12591CC004C005C006C00790001A2C
:10367800E0FCA3E0FDA3E0FEA3E0FF12591CA804B0
:10368800A905AA06AB07D007D006D005D0041219A1
:1036980057A804A905AA06AB07D007D006D005D0BD
:1036A800041218669001A0122011900190E0FCA36A
:1036B800E0FDA3E0FEA3E0FF125906C004C005C068
:1036C80006C007900016E0FCA3E0FDA3E0FEA3E01F
:1036D800FF12591CA804A905AA06AB07D007D006F3
:1036E800D005D004121957C004C005C006C0079001
:1036F80001A0E0FCA3E0FDA3E0FEA3E0FF9001A091
:10370800E0F8A3E0F9A3E0FAA3E0FB121957A80434
:10371800A905AA06AB077F007E007D807C3F1218B2
:103728006212665BA804A905AA06AB07D007D006F3
:10373800D005D004121A609001A01220119001A0A7
:10374800E0FCA3E0FDA3E0FEA3E0FFC004C005C0C9
:1037580006C0079001A4E0FCA3E0FDA3E0FEA3E0FF
:10376800FF9000E8122011D007D006D005D004122F
:1037780068E7900182E0FBA3E0FAA3E0F9121F9F3B
:10378800900182E0FBA3E0FAA3E0F9121F7F7B001F
:103798007A0079007800121AFD6030402E9001827C
:1037A800E0FBA3E0FAA3E0F9C003C002C001121FC6
:1037B8007F9001E6E0F8A3E0F9A3E0FAA3E0FB12AA
:0B37C8001866D001D002D003121F9F32
:0137D30022D3
:1065AB00323B171C0205006400640001000007A3C6
:1065BB0000870384006407080384068205690007CB
:1065CB0000020009003B003B0017001C000C00639D
:1065DB0000C700C70002000A0E0F03840E0F0384CE
:1065EB000E0F07080E0F070800080005000E00002D
:1065FB00000000000001000100000001000100008C
:10660B00000000000000000000000000000000007F
:10661B000000000000000000000000030000000369
:10662B00000200030002000300030002000300024B
:10663B00000300000003000100030002000300023E
:0C664B0000030003000200030002000333
:066C5200C119C11BC11AAB
:106A1E009000107432F0900011743BF090001274DC
:106A2E0017F0900013741CF09000147402F0900094
:106A3E00157405F0124F41757900757A00D3E57A19
:106A4E00940EE57964809480503CE57A25E0FFE56C
:106A5E007933FE74B12FF58274653EF583E493FCB1
:106A6E00740193FDE57A25E0FFE57933FE74222F5C
:106A7E00F58274003EF583ECF0A3EDF0057AE57A2D
:106A8E007002057980B7125045900068E4F0A3E4D7
:106A9E00F090006AE4F0A3E4F090006CE4F0A3E45C
:056AAE00F01250672208
:10413B0090003FE0F574D3E57464809482400BC328
:10414B00E574648094865002C219E5A064FFFFEF0A
:10415B005407F576E5766006C29CC2988002D29C25
:10416B00E5765406FFEF60270578E578D3940A408F
:10417B000F75750AC3E57464809486500375780ACD
:10418B00E578D39414400E757564757814800675B4
:10419B007800757501AF74EF3395E0FEEF25E0FF06
:1041AB00EE33FE74F92FF58274653EF583E493F5D7
:1041BB0072740193F573AF74EF3395E0FEEF25E066
:1041CB00FFEE33FE74CF2FF58274653EF583E493D7
:1041DB00F570740193F571E5746403706B900015C1
:1041EB00E0FFEF75F004121E39AFF0EF602E900078
:1041FB0014E0FFEF3395E0FEEF25E0FFEE33FE74A6
:10420B00232FF58274663EF583E493FE740193FFCE
:10421B00EF2571F571EE3570F570802C900014E080
:10422B00FFEF3395E0FEEF25E0FFEE33FE743D2FFD
:10423B00F58274663EF583E493FE740193FFEF25DC
:10424B0071F571EE3570F570E576B40110900028BC
:10425B00E0FEA3E0FFEF4E70040577800375770057
:10426B00E577C394144008757700A219B39219D35C
:10427B00E57664809481500302452AC3E57464801B
:10428B0094864003024350124F96E57664047055B2
:10429B00AF74EF3395E0FE74102FF58274003EF58A
:1042AB0083E02575F0AF74EF3395E0FE74102FF5B6
:1042BB008274003EF583E0FFEF3395E0FED3EF957C
:1042CB0071E5706480F8EE6480984016AF73AE743D
:1042DB00EEFD3395E0FC74102DF58274003CF583F4
:1042EB00EFF0124F41E5766402705AAF74EF3395DD
:1042FB00E0FE74102FF58274003EF583E0FFC3EFF0
:10430B009575FFEFF0AF74EF3395E0FE74102FF55A
:10431B008274003EF583E0FFEF3395E0FEC3EF952B
:10432B0073E5726480F8EE6480985016AF71AE74CA
:10433B00EEFD3395E0FC74102DF58274003CF58393
:10434B00EFF0124F41C3E57464809486500302442E
:10435B006C74FA2574F574E57664047072AF75EFBE
:10436B00FD7C00AF74EF3395E0FEEF25E0FFEE33FD
:10437B00FE74222FF58274003EF583EC8DF0121E35
:10438B00FBAF74EF3395E0FEEF25E0FFEE33FE74E9
:10439B00222FF58274003EF583E0FEA3E0FFD3EFFE
:1043AB009571E5706480F8EE648098401FAF74EFF0
:1043BB003395E0FEEF25E0FFEE33FE74222FF582FE
:1043CB0074003EF583E572F0A3E573F0125045E5FA
:1043DB007664026003024466AF74EF3395E0FEEF40
:1043EB0025E0FFEE33FE74222FF58274003EF58339
:1043FB00C083C082E0FEA3E0FFAD757C00C3EF9DE0
:10440B00FFEE9CFED082D083EEF0A3EFF0AF74EF03
:10441B003395E0FEEF25E0FFEE33FE74222FF5829D
:10442B0074003EF583E0FEA3E0FFC3EF9573E572E6
:10443B006480F8EE648098501FAF74EF3395E0FE04
:10444B00EF25E0FFEE33FE74222FF58274003EF56C
:10445B0083E570F0A3E571F012504574062574F5F1
:10446B0074900028E0FEA3E0FFEF4E705CE576B49D
:10447B000526301B230574AF74D3EF6480949340EF
:10448B0003757400C21BAF74EF3395E0FE90003ED2
:10449B00EEF0A3EFF0125045E5766403600302459E
:1044AB002A301B7B1574AF74C3EF64809480500368
:1044BB00757413C21BAF74EF3395E0FE90003EEEA4
:1044CB00F0A3EFF01250458056E576B40526301B6D
:1044DB00230574AF74D3EF6480949240037574001A
:1044EB00C21BAF74EF3395E0FE90003EEEF0A3EFEE
:1044FB00F0125045E576B40326301B231574AF74C8
:10450B00C3EF648094805003757412C21BAF74EFB9
:10451B003395E0FE90003EEEF0A3EFF0125045E530
:10452B0076B40102D21BE5765406FFEF60109000C3
:10453B003EE0FEA3E0FFEF64094E7002C20F900253
:10454B0001E0FEA3E0FF900028E0FCA3E0FDED6F8F
:10455B007002EC6E6002C20F900028E0FEA3E0FF39
:10456B00900201EEF0A3EFF030A302D21A20A30ABF
:0A457B00301A07C21AA20FB3920F04
:014585002213
:104F41001250B074A01250C874021250C8900010D0
:104F51007C03E01250891250C8A3DCF6E01250899C
:104F6100F5F0A3A3E0030354C045F01250C890002C
:104F710014E01250891250C8C2B41250A31250B09A
:104F810074A01250C874F01250C8A3E01250C8C2E5
:104F9100B41250A3221250B074A01250C87402125D
:104FA10050C81250B074A0041250C8900010125092
:104FB100ED125091F0A31251001250ED125091F0E8
:104FC100A31251001250ED125091F0A31251001290
:104FD10050EDFB543F125091F0A31251001250EDCD
:104FE100FA541F125091F0EB23235403FD1250FA8F
:104FF100C2B41250A31250B074A01250C874F0126F
:1050010050C81250B074A0041250C81250EDFB5495
:1050110003C39D2405838007030201000302012BC2
:10502100A3F0F5F01250FAC2B41250A31250B074AA
:10503100A01250C874F01250C8E5F01250C8C2B4A2
:105041001250A3227AA07B807C1E90002212514034
:10505100227AA07B80125108ED900022F07AA0A361
:105061007C1D125175227AA07BD07C1090006812B1
:105071005140227AA07BD0125108ED900068F07A5D
:01508100A08E
:10508200A37C0F1251752275F00A84C425F022C048
:10509200E0C4540F75F00AA4F5F0D0E0540F25F0E7
:1050A2002200D2B5000000D2B4000000002212504B
:1050B200A3C2B4000000C2B500000022D2B50000B5
:1050C20000C2B50000227E083392B41250BEDEF850
:1050D20033D2B40000A2B450040000A2B41250BEF5
:1050E200400122C2B400001250A3227E08A2B433AF
:1050F200001250BEDEF7C322D2B41250BE22C2B496
:105102001250BED2B4221250B0EA1250C8EB125062
:10511200C81250B0EA041250C81250EDFD1250FAF3
:10512200C2B41250A3221250B0EA1250C8EB12506D
:10513200C8E61250C808DCF9C2B41250A3221250B9
:10514200B0EA1250C8EB1250C8E01250C8A3DCF902
:10515200C2B41250A3221250B0EA041250C8800303
:105162001251001250EDF608DCF61250FAC2B412D7
:1051720050A3221250B0EA041250C8800312510008
:0C5182001250EDF0A3DCF61250FAC2B49B
:04518E001250A322F6
:104C4E00202020202531642E25303264202530325C
:104C5E0062753A25303262753A25303262752020FF
:104C6E00202000202020202532642E25316420258E
:104C7E00303262753A25303262753A2530326275BD
:104C8E002020202000253033642E2531642020255D
:104C9E003032642E25316420415A2F454C3120206C
:104CAE002000253033642E253164202025303264D7
:104CBE002E25316420415A2F454C322020200025CC
:104CCE003033642E2531642020253032642E253178
:104CDE00642052412F444543202020002530336468
:104CEE002E2531645720253032642E2531644E2016
:104CFE004C4F2F4C41202020002530326275202051
:104D0E00202530326275202025303262753A2530EA
:104D1E003262753A2530326275202020200025300F
:104D2E00352E31662020253032642E253164202028
:104D3E00202020202025303264202000202B2530FA
:104D4E0031642E2530316420202B253031642E2500
:104D5E0030316420434F52202053545020002D2DCB
:104D6E002D2D2D2D2D2D2D2D2D202020202020538D
:104D7E0054502000253033642E25316420202530F8
:104D8E0032642E25316420414E5420202531642E6C
:104D9E002531642000202020204F20452035204A38
:104DAE002046204C202020202000202020202020C3
:104DBE002020454D4520202020202020202000208E
:104DCE00416E74656E6E6120436F6E74726F6C6CA3
:104DDE0065722000202020202020207620372E31C2
:104DEE002020202020202020002020204A414E4636
:104DFE0045424D41524150524D41594A554E4A55E8
:104E0E004C4155475345504F43544E4F56444543DE
:104E1E00004D4F4F4E202053554E202020434153DE
:104E2E0053494F4359474E55535341474954545490
:104E3E0041555255534C454F20202041515541521A
:104E4E002E52412F444543415A2F454C32415A2F41
:104E5E00454C3100326D3A37303A32333A31333ACB
:104E6E0036636D313047002053534920313062692B
:104E7E0074283732302920202020202053534931E6
:104E8E0031626974283138303029202020202020CA
:104E9E005353493132626974283336303029202019
:104EAE00202020205353495F6772617928343039AE
:104EBE00362920202020202041322D532D53203101
:104ECE0032206269742020202020204D414232354C
:104EDE005F31306269743130323420202020204D11
:104EEE00414232355F3131626974323034382020BC
:104EFE002020204D414232355F31326269743430A8
:104F0E00393620202020204D414232385F31326226
:104F1E006974343039362020202020000F0C09010E
:104F2E000306171D664C03090309030903095601FD
:034F3E0001020469
:10002E00E57664016003125C2E201403020663C29F
:10003E001430190C900028E0FEA3E0FFEF4E601183
:10004E0090003EE0FEA3E0FFEF64134E600302015A
:10005E00FB90003CE0FEA3E0FFC3EF9404EE64804F
:10006E0094804003020108AF1CAE1B126D83EF2477
:10007E0005FFEE3400FE7C007D0A121EC59000E0E6
:10008E00EEF0A3EFF07B017A007980C003C002C0CE
:10009E00017BFF7A4C794E9000F3EBF0A3EAF0A3CC
:1000AE00E9F09000E0E0FEA3E0FF7C007D64121E0C
:1000BE00C59000F6EEF0A3EFF09000E0E0FEA3E0B6
:1000CE00FF7C007D64121EC59000F8ECF0A3EDF0ED
:1000DE00900012E0FF9000FAEFF0900011E0FF9018
:1000EE0000FBEFF0900010E0FF9000FCEFF0D0016D
:1000FE00D002D003123D1D020198AF1CAE1B126D33
:10010E0083EF2432FFEE3400FE7C007D64121EC5A8
:10011E009000E0EEF0A3EFF07B017A007980C0034F
:10012E00C002C0017BFF7A4C79719000F3EBF0A313
:10013E00EAF0A3E9F09000E0E0FEA3E0FF7C007D92
:10014E000A121EC59000F6EEF0A3EFF09000E0E06C
:10015E00FEA3E0FF7C007D0A121EC59000F8ECF0B5
:10016E00A3EDF0900012E0FF9000FAEFF090001176
:10017E00E0FF9000FBEFF0900010E0FF9000FCEF2E
:10018E00F0D001D002D003123D1D751500D3E51538
:10019E00648094825042AF1590003DE0FE75F003EE
:1001AE00EEA4F58285F083E5822FF582E43583F5A2
:1001BE0083E5822462F582E583344EF583E493FF72
:1001CE00AE15EEFD3395E0FC74802DF58274003C87
:1001DE00F583EFF0051580B5C3E51B648094804070
:1001EE00030205F3900083742DF00205F390003E98
:1001FE00E0FEA3E0FFEF640A4E601190003EE0FEC9
:10020E00A3E0FFEF640B4E600302029F7B017A00B6
:10021E007980C003C002C0017BFF7A4C79939000B5
:10022E00F3EBF0A3EAF0A3E9F090002AE0FEA3E0DE
:10023E00FF7C007D0A121EC59000F6EEF0A3EFF0D3
:10024E0090002AE0FEA3E0FF7C007D0A121EC590FE
:10025E0000F8ECF0A3EDF090002CE0FEA3E0FF7CA4
:10026E00007D0A121EC59000FAEEF0A3EFF090008A
:10027E002CE0FEA3E0FF7C007D0A121EC59000FC60
:10028E00ECF0A3EDF0D001D002D003123D1D02051B
:10029E00F390003EE0FEA3E0FFEF640C4E60119081
:1002AE00003EE0FEA3E0FFEF640D4E600302034349
:1002BE007B017A007980C003C002C0017BFF7A4CBB
:1002CE0079B09000F3EBF0A3EAF0A3E9F090002EE2
:1002DE00E0FEA3E0FF7C007D0A121EC59000F6EE44
:1002EE00F0A3EFF090002EE0FEA3E0FF7C007D0A6D
:1002FE00121EC59000F8ECF0A3EDF0900030E0FE79
:10030E00A3E0FF7C007D0A121EC59000FAEEF0A35A
:10031E00EFF0900030E0FEA3E0FF7C007D0A121E9D
:10032E00C59000FCECF0A3EDF0D001D002D003128A
:10033E003D1D0205F390003EE0FEA3E0FFEF640ECC
:10034E004E601190003EE0FEA3E0FFEF640F4E60A2
:10035E0003020426900034E0FEA3E0FFEF247CFFAE
:10036E00EE34FCFE90007CEEF0A3EFF090007CE00B
:10037E00FEA3E0FF126D837C007D0A121EC5C0062F
:10038E00C00790007CE0FEA3E0FF126D837C007D31
:10039E000A121EC59000FCECF0A3EDF0D007D006BB
:1003AE009000FAEEF0A3EFF07B017A007980C003A3
:1003BE00C002C0017BFF7A4C79CD9000F3EBF0A325
:1003CE00EAF0A3E9F0900032E0FEA3E0FF7C007DAE
:1003DE000A121EC59000F6EEF0A3EFF0900032E088
:1003EE00FEA3E0FF7C007D0A121EC59000F8ECF023
:1003FE00A3EDF0D001D002D003123D1D90007CE0A1
:10040E00FEA3E0FFC3EE6480948040030205F390E8
:10041E000086742DF00205F390003EE0FEA3E0FF8F
:10042E00EF64104E601190003EE0FEA3E0FFEF641B
:10043E00114E600302054D900036E0FEA3E0FFEF83
:10044E0024F8FFEE34F8FE90007EEEF0A3EFF0906D
:10045E000038E0FEA3E0FFEF247CFFEE34FCFE90BC
:10046E00007CEEF0A3EFF090007EE0FEA3E0FF1222
:10047E006D837C007D0A121EC5C006C00790007EEB
:10048E00E0FEA3E0FF126D837C007D0A121EC5C044
:10049E0004C00590007CE0FEA3E0FF126D837C009B
:1004AE007D0A121EC5C006C00790007CE0FEA3E0C8
:1004BE00FF126D837C007D0A121EC59000FCECF0CD
:1004CE00A3EDF0D007D0069000FAEEF0A3EFF0D037
:1004DE0005D0049000F8ECF0A3EDF0D007D0069014
:1004EE0000F6EEF0A3EFF07B017A007980C003C036
:1004FE0002C0017BFF7A4C79EA9000F3EBF0A3EA9D
:10050E00F0A3E9F0D001D002D003123D1D90007E81
:10051E00E0FEA3E0FFC3EE64809480500690008559
:10052E007445F090007CE0FEA3E0FFC3EE6480947F
:10053E008040030205F390008B7453F00205F37BA9
:10054E00017A007980C003C002C0017BFF7A4D7929
:10055E00079000F3EBF0A3EAF0A3E9F0900013E0AC
:10056E00FF9000F6EFF0900015E0FF9000F7EFF02F
:10057E00900012E0FF9000F8EFF0900011E0FF9075
:10058E0000F9EFF0900010E0FF9000FAEFF0D001CC
:10059E00D002D003123D1D751500D3E5156480946D
:1005AE00825042AF15900014E0FE75F003EEA4F5F4
:1005BE008285F083E5822FF582E43583F583E5822B
:1005CE0024F7F582E583344DF583E493FFAE15EE03
:1005DE00FD3395E0FC74822DF58274003CF583EFBB
:1005EE00F0051580B5900028E0FEA3E0FFC3EF9460
:1005FE0002EE64809480503290003EE0FEA3E0FF55
:10060E00C3EF940AEE64809480401390003EE0FEA7
:10061E00A3E0FFD3EF9411EE64809480400C900021
:10062E00927444F09000937445F07F00125C407514
:10063E001500D3E51564809493501AAF15EF3395DA
:10064E00E0FE74802FF58274003EF583E0FF125CAD
:10065E0007051580DD201503020879C21590003EAE
:10066E00E0FEA3E0FFC3EF940AEE64809480401591
:10067E0090003EE0FEA3E0FFD3EF9411EE64809471
:10068E00805002C2199001E2E0F8A3E0F9A3E0FA6B
:10069E00A3E0FB900004E0FCA3E0FDA3E0FEA3E0DA
:1006AE00FF121A60126DEA7B007A007920784112EF
:1006BE0019577B007A007900783F121866121BB921
:1006CE0090007CEEF0A3EFF09001E2E0F8A3E0F9E9
:1006DE00A3E0FAA3E0FB900078E0FCA3E0FDA3E02A
:1006EE00FEA3E0FF121A60126DEA7B007A00790019
:1006FE00783F121866121BB99000E2EEF0A3EFF0ED
:10070E007B017A007998C003C002C0017BFF7A4D4D
:10071E00792C9000F3EBF0A3EAF0A3E9F09001E25C
:10072E00E0F8A3E0F9A3E0FAA3E0FB90000CE0FCF4
:10073E00A3E0FDA3E0FEA3E0FF121A609000F61204
:10074E00201190007CE0FEA3E0FF7C007D0A121ECB
:10075E00C59000FAEEF0A3EFF090007CE0FEA3E06F
:10076E00FF7C007D0A121EC59000FCECF0A3EDF09C
:10077E009000E2E0FEA3E0FF9000FEEEF0A3EFF0AB
:10078E00D001D002D003123D1D7F007E007D007C83
:10079E0000900004E0F8A3E0F9A3E0FAA3E0FB1256
:1007AE001AFD500690009E742DF0751500D3E515B8
:1007BE00648094855042AF15900029E0FE75F006D6
:1007CE00EEA4F58285F083E5822FF582E43583F57C
:1007DE0083E582241FF582E583344EF583E493FF8F
:1007EE00AE15EEFD3395E0FC74A42DF58274003C3D
:1007FE00F583EFF0051580B5900028E0FEA3E0FF2D
:10080E00C3EF9402EE64809480400E9000AA742090
:10081E00F09000AB7420F080217F007E007D007C84
:10082E0000900078E0F8A3E0F9A3E0FAA3E0FB1251
:10083E001AFD50069000A9742DF0E5766401602B28
:10084E007F40125C40751500D3E51564809493507B
:10085E001AAF15EF3395E0FE74982FF58274003EB3
:10086E00F583E0FF125C07051580DD2016030209F3
:10087E00CAC216900022E0FEA3E0FFEF249CFFEE1A
:10088E0034FFFE126D8390007EEEF0A3EFF0900029
:10089E0024E0FEA3E0FFEF249CFFEE34FFFE126D7A
:1008AE008390007CEEF0A3EFF03010030209417B41
:1008BE00017A0079B0C003C002C0017BFF7A4D7986
:1008CE004A9000F3EBF0A3EAF0A3E9F090007EE08B
:1008DE00FEA3E0FF7C007D0A121EC59000F6EEF02E
:1008EE00A3EFF090007EE0FEA3E0FF7C007D0A12F5
:1008FE001EC59000F8ECF0A3EDF090007CE0FEA396
:10090E00E0FF7C007D0A121EC59000FAEEF0A3EF08
:10091E00F090007CE0FEA3E0FF7C007D0A121EC575
:10092E009000FCECF0A3EDF0D001D002D003123D0C
:10093E001D80267B017A0079B0C003C002C0017B06
:10094E00FF7A4D796C9000F3EBF0A3EAF0A3E9F097
:10095E00D001D002D003123D1D900022E0FEA3E094
:10096E00FFC3EF9464EE6480948050069000B174DF
:10097E002DF0900024E0FEA3E0FFC3EF9464EE643C
:10098E0080948050069000B7742DF0E57664016077
:10099E002B7F14125C40751500D3E515648094937B
:1009AE00501AAF15EF3395E0FE74B02FF582740038
:1009BE003EF583E0FF125C07051580DD201703026C
:1009CE000BCCC217900027E0FFEF904F3E93FFEF46
:1009DE003395E0FEAC66AD67121EB38E4A8F4BAFF9
:1009EE0048AE47126D837C007D0A121EC5C006C03C
:1009FE0007AF48AE47126D837C007D0A121EC5906C
:100A0E0000FCECF0A3EDF0D007D0069000FAEEF06B
:100A1E00A3EFF07B017A0079C8C003C002C0017B4E
:100A2E00FF7A4D79829000F3EBF0A3EAF0A3E9F0A0
:100A3E00AE4DAF4E7C007D0A121EC59000F6EEF054
:100A4E00A3EFF0AE4DAF4E7C007D0A121EC5900096
:100A5E00F8ECF0A3EDF0AE4AAF4B7C007D0A121E0F
:100A6E00C59000FEEEF0A3EFF0AE4AAF4B7C007DDA
:100A7E000A121EC5900100ECF0A3EDF0D001D002D9
:100A8E00D003123D1DC3E54764809480500690004C
:100A9E00CE742DF0A21CB3921CE508540CFFEFB4DB
:100AAE000808201C059000D8E4F0E508540CFFEF70
:100ABE00B40409201C069000D87401F0E508540C0B
:100ACE00FFEFB40C09300F069000D8742AF0E50839
:100ADE005403FFEFB40209301C069000D77402F0E5
:100AEE00E5085403FFEFB40109301C069000D774DB
:100AFE0003F0E5085403FFEFB40309300F0690002E
:100B0E00D7742AF090003EE0FEA3E0FFEF64124E91
:100B1E006003020BA1751500D3E515648094935004
:100B2E0042AF1590003BE0FE75F014EEA4F5828501
:100B3E00F083E5822FF582E43583F583E582247513
:100B4E00F582E583344EF583E493FFAE15EEFD3367
:100B5E0095E0FC74C82DF58274003CF583EFF0052A
:100B6E001580B5AE4AAF4B7C007D0A121EC5EF2430
:100B7E0030FF9000D9EFF09000DA742EF0AE4AAF4D
:100B8E004B7C007D0A121EC5AF05EF2430FF90008E
:100B9E00DBEFF07F54125C40751500D3E5156480D1
:100BAE009493501AAF15EF3395E0FE74C82FF5826B
:100BBE0074003EF583E0FF125C07051580DDE576D7
:100BCE00B4011490003FE0FFEF904F2A93FF125CA8
:100BDE0040125C25125C37301803020D2F7B017A10
:100BEE00007980C003C002C0017BFF7A4D79A390CB
:100BFE0000F3EBF0A3EAF0A3E9F0D001D002D003AA
:100C0E00123D1D7B017A007998C003C002C0017BA2
:100C1E00FF7A4D79B89000F3EBF0A3EAF0A3E9F078
:100C2E00D001D002D003123D1D7B017A0079B0C0F5
:100C3E0003C002C0017BFF7A4D79CD9000F3EBF03B
:100C4E00A3EAF0A3E9F0D001D002D003123D1D7B40
:100C5E00017A0079C8C003C002C0017BFF7A4D79CA
:100C6E00E29000F3EBF0A3EAF0A3E9F0D001D0029A
:100C7E00D003123D1D7F00125C40751500D3E515A3
:100C8E0064809493501AAF15EF3395E0FE74802F65
:100C9E00F58274003EF583E0FF125C07051580DDDA
:100CAE007F40125C40751500D3E515648094935017
:100CBE001AAF15EF3395E0FE74982FF58274003E4F
:100CCE00F583E0FF125C07051580DD7F14125C4092
:100CDE00751500D3E51564809493501AAF15EF3354
:100CEE0095E0FE74B02FF58274003EF583E0FF129E
:100CFE005C07051580DD7F54125C40751500D3E549
:100D0E001564809493501AAF15EF3395E0FE74C8B6
:100D1E002FF58274003EF583E0FF125C0705158007
:020D2E00DD22C4
:106C5800015100014F00015000014900C10FC10C52
:0A6C6800C10BC10EC110C10DC11116
:106D9500752400D3E524648094A75004052480F36A
:016DA50022CB
:106DA600752500D3E525648094935004052580F36A
:016DB60022BA
:106DB700752600D3E5266480949E5004052680F34B
:016DC70022A9
:106DC800752700D3E5276480949E5004052780F337
:016DD8002298
:106DD900752800D3E5286480949E5004052880F323
:016DE9002287
:105FBD00C290126D95752E1F752D00E52DD394078A
:105FCD005011E52EC313F52EA2D79290126D9505A3
:105FDD002D80E8D290126D95D292752903752AE81D
:105FED00752E00309110E52A152A7002152914FF1F
:105FFD00AE29EF4E70ED126DA6752D00E52DD394E3
:10600D00075013126D95E52EC313F52E30910343F2
:10601D002E80052D80E6126D95AF2E7E00EF752C2E
:10602D0000F52B752903752AE8752E00309110E5C2
:10603D002A152A7002152914FFAE29EF4E70ED12A4
:10604D006DA6752D00E52DD394075013126D95E5B2
:10605D002EC313F52E309103432E80052D80E612AD
:10606D006D95AF2E7E00EF252CF52CEE352BF52BF7
:10607D00C3E52B648094805006752B00752C00D3DE
:10608D00E52C940FE52B6480948E4006752B0E75D0
:10609D002C0FC29220B20DC3740F952CF52C740EDB
:0860AD00952BF52BAE2BAF2C57
:0160B50022C8
:10629400C294126D9575341F753300E533D394079A
:1062A4005011E534C313F534A2D79294126D9505B9
:1062B4003380E8D294126D95D296752F037530E829
:1062C400753400309510E53015307002152F14FF29
:1062D400AE2FEF4E70ED126DA6753300E533D394F7
:1062E400075013126D95E534C313F5343095034309
:1062F4003480053380E6126D95AF347E00EF75323D
:1063040000F531752F037530E8753400309510E5CC
:106314003015307002152F14FFAE2FEF4E70ED12B2
:106324006DA6753300E533D394075013126D95E5CC
:1063340034C313F534309503433480053380E612B7
:106344006D95AF347E00EF2532F532EE3531F531FF
:10635400C3E531648094805006753100753200D3F2
:10636400E532940FE5316480948E400675310E75E4
:08637400320FC296AE31AF32C8
:01637C0022FE
:10000E00125FBD8E4D8F4E1262948E478F4875666D
:05001E000075670122DE
:1067A800D290D294D291D295756C00756D007568AF
:1067B80000756900753500D3E535648094895049C2
:1067C800126DB7C290C294126DB7C3E53564809458
:1067D800895004D290D294E56D256DF56DE56C3540
:1067E8006CF56CE5692569F569E5683568F5682033
:1067F8009108056DE56D7002056C2095080569E541
:106808006970020568053580AEC290C2947566004D
:10681800756705AE6CAF6D7C007D05121EB38E4D9D
:106828008F4E20B20DC3740B954EF54E740E954DD8
:10683800F54DAE68AF697C007D05121EB38E478F9B
:016848004807
:01684900222C
:10698400D290D294D291D295756C00756D007568D1
:1069940000756900753600D3E5366480948A5049E1
:1069A400126DB7C290C294126DB7C3E53664809479
:1069B4008A5004D290D294E56D256DF56DE56C3561
:1069C4006CF56CE5692569F569E5683568F5682055
:1069D4009108056DE56D7002056C2095080569E563
:1069E4006970020568053680AEC290C2947566006F
:1069F400756702E56D25E0F54EE56C33F54D20B283
:106A04000DC3740E954EF54E740E954DF54DE56916
:096A140025E0F548E56833F5477B
:016A1D002256
:106B4400D290D294D291D295756C00756D0075680F
:106B540000756900753700D3E5376480948B50491C
:106B6400126DB7C290C294126DB7C3E537648094B6
:106B74008B5004D290D294E56D256DF56DE56C359E
:106B84006CF56CE5692569F569E5683568F5682093
:106B94009108056DE56D7002056C2095080569E5A1
:106BA4006970020568053780AEC290C294756600AC
:106BB400756701856C4D856D4E20B20DC3740F95BC
:0F6BC4004EF54E740E954DF54D85684785694821
:016BD300229F
:105C8500D292D291756C00756D00126DC875380091
:105C9500D3E5386480948F5025D290126DC8C29098
:105CA500126DC8E56D256DF56DE56C356CF56C20EF
:105CB5009108056DE56D7002056C053880D2C290BE
:105CC500C292E56DAE6C7806CEC313CE13D8F9F546
:105CD5006D8E6CAC6CAD6DE4121B807B007A007927
:105CE5003478441219577B007A0079807844121A67
:105CF50060121BB97C007D05121EB38E4D8F4E20A0
:105D0500B20DC3740B954EF54E740E954DF54D12AF
:105D15006DC8756600756705D296D295756800756C
:105D25006900126DC8753800D3E5386480948F50CA
:105D350025D294126DC8C294126DC8E5692569F51E
:105D450069E5683568F5682095080569E5697002B3
:105D55000568053880D2C294C296E569AE687806B2
:105D6500CEC313CE13D8F9F5698E68AC68AD69E476
:105D7500121B807B007A00793478441219577B0016
:105D85007A0079807844121A60121BB97C007D056F
:075D9500121EB38E478F4878
:015D9C0022E4
:105D9D00D292D291756C00756D00126DC875390077
:105DAD00D3E5396480948F5025D290126DC8C2907E
:105DBD00126DC8E56D256DF56DE56C356CF56C20D6
:105DCD009108056DE56D7002056C053980D2C290A4
:105DDD00C292E56DAE6C7805CEC313CE13D8F9F52E
:105DED006D8E6CAC6CAD6DE4121B807B007A00790E
:105DFD00E178441219577B007A0079007845121A20
:105E0D0060121BB9EF25E0F54EEE33F54D20B20DC6
:105E1D00C3740E954EF54E740E954DF54D126DC81D
:105E2D00756600756702D296D29575680075690022
:105E3D00126DC8753900D3E5396480948F5025D221
:105E4D0094126DC8C294126DC8E5692569F569E5AE
:105E5D00683568F5682095080569E569700205687B
:105E6D00053980D2C294C296E569AE687805CEC375
:105E7D0013CE13D8F9F5698E68AC68AD69E4121BC1
:105E8D00807B007A0079E178441219577B007A0003
:105E9D0079007845121A60121BB9EF25E0F548EE2E
:035EAD0033F54783
:015EB00022CF
:105EB100D292D291756C00756D00126DC8753A0061
:105EC100D3E53A6480948F5025D290126DC8C29068
:105ED100126DC8E56D256DF56DE56C356CF56C20C1
:105EE1009108056DE56D7002056C053A80D2C2908E
:105EF100C292E56CC4F854F0C868F56CE56DC45401
:105F01000F48F56DAC6CAD6DE4121B807B007A001F
:105F1100796178451219577B007A007980784512AA
:105F21001A60121BB98E4D8F4E20B20DC3740F959E
:105F31004EF54E740E954DF54D126DC87566007592
:105F41006701D296D295756800756900126DC875A2
:105F51003A00D3E53A6480948F5025D294126DC8EB
:105F6100C294126DC8E5692569F569E5683568F57A
:105F7100682095080569E56970020568053A80D2CF
:105F8100C294C296E568C4F854F0C868F568E5693A
:105F9100C4540F48F569AC68AD69E4121B807B00FD
:105FA1007A00796178451219577B007A00798078F7
:0B5FB10045121A60121BB98E478F4882
:015FBC0022C2
:10571A00D292D291756C00756D00126DD9753B00ED
:10572A00D3E53B6480948F5025D290126DD9C290F4
:10573A00126DD9E56D256DF56DE56C356CF56C204E
:10574A009108056DE56D7002056C053B80D2C2902B
:10575A00C292E56CC4F854F0C868F56CE56DC4549F
:10576A000F48F56DD3E56D9559E56C955840188548
:10577A006C62856D63856C58856D59E56D24FFF5FE
:10578A0057E56C34FFF556C3E56D9557E56C9556AC
:10579A00501EE56D2401F563E56C3400F562856CF5
:1057AA0056856D57E56D2401F559E56C3400F558B9
:1057BA00AC62AD63EC121B807B007A00796178459C
:1057CA001219577B007A0079807845121A60121BE9
:1057DA00B98E4D8F4E20B20DC3740F954EF54E748F
:1057EA000E954DF54D126DC8756600756701D29616
:1057FA00D295756800756900126DD9753B00D3E5BD
:10580A003B6480948F5025D294126DD9C294126D44
:10581A00D9E5692569F569E5683568F56820950867
:10582A000569E56970020568053B80D2C294C29693
:10583A00E568C4F854F0C868F568E569C4540F48C7
:10584A00F569D3E5699555E5689554401885685E0C
:10585A0085695F856854856955E56924FFF553E5CF
:10586A006834FFF552C3E5699553E5689552501EB1
:10587A00E5692401F55FE5683400F55E85685285BF
:10588A006953E5692401F555E5683400F554AC5EC1
:10589A00AD5FEC121B807B007A00796178451219A2
:1058AA00577B007A0079807845121A60121BB98EEC
:0358BA00478F48CD
:0158BD0022C8
:1061A600D290D294D291D295756C00756D007568B7
:1061B60000756900753C00D3E53C6480948B5053B0
:1061C600C290C294753D00D3E53D6480948250042C
:1061D600053D80F3C3E53C6480948B5004D290D295
:1061E60094E56D256DF56DE56C356CF56CE5692509
:1061F60069F569E5683568F568209108056DE56D0E
:106206007002056C2095080569E569700205680548
:106216003C80A4C290C294756600756701AF6DAEEE
:106226006C126D6B8E6C8F6DAF69AE68126D6B8E76
:10623600688F69AC6CAD6DE4121B807B007A0079C7
:106246006178451219577B007A0079807845121AD1
:1062560060121BB98E4D8F4E20B20DC3740F954E32
:10626600F54E740E954DF54DAC68AD69E4121B8084
:106276007B007A00796178451219577B007A00799C
:0D628600807845121A60121BB98E478F48B0
:0162930022E8
:1037D400E54C64326003300D61C3E56F954EF561CD
:1037E400E56E954DF560C374089548FF74079547D9
:1037F400FE126D83C374849FFF74039EFEC3E56B46
:103804009FF55BE56A9EF55AC3E5489408E547646D
:10381400809487400BC3E4955BF55BE4955AF55AB5
:10382400C210C20E900068E560F0A3E561F090005C
:103834006AE55AF0A3E55BF0C20D20101B20B30328
:10384400300E03301112D210D20E90006CE4F0A3AB
:103854007401F0125067C21130101D20B303300EF2
:1038640003301114C210D20E12505290006CE4F0C6
:10387400A3E4F0125067C21120B304054C8005750F
:103884004C00C20E301074E561254EF54EE56035EE
:103894004DF54DD3E54E940FE54D6480948E400C68
:1038A40074F0254EF54E74F1354DF54DC3E54D6478
:1038B400809480500C7410254EF54E740E354DF5E1
:1038C4004DE55B2548F548E55A3547F547D3E548C6
:1038D400940FE5476480948E400C74F02548F548B5
:1038E40074F13547F547C3E54764809480500C7400
:1038F400102548F548740E3547F547C374089548B4
:10390400FF74079547FE126D83C374849FF5487452
:10391400039EF547E56F24F8F55DE56E34F8F55C34
:10392400E54E24F8F565E54D34F8F564C3E55C64CB
:10393400809480500C7410255DF55D740E355CF533
:103944005CC3E56464809480500C74102565F5654F
:10395400740E3564F56430105A900038E0FEA3E02C
:10396400FFC3EF9484EE64809483400FC3E56F95A6
:103974004EF53FE56E954DF53E800DC3E55D9565CD
:10398400F53FE55C9564F53ED3E56B9400E56A6428
:103994008094804010C3E56B9548F541E56A9547EE
:1039A400F540023A5FC3E49548F541E49547F54094
:1039B400023A5F900038E0FEA3E0FFC3EF9484EE88
:1039C400648094834025900022E0FEA3E0FFE56F2D
:1039D4002FFFE56E3EFEEF249CFFEE34FFFEC3EFA7
:1039E400954EF53FEE954DF53E8023900022E0FE86
:1039F400A3E0FFE55D2FFFE55C3EFEEF249CFFEEB8
:103A040034FFFEC3EF9565F53FEE9564F53ED3E5CF
:103A14006B9400E56A648094804025900024E0FE65
:103A2400A3E0FFE56B2FFFE56A3EFEEF249CFFEE6B
:103A340034FFFEC3EF9548F541EE9547F540801BF2
:103A4400900024E0FEA3E0FFEF249CFFEE34FFFE91
:103A5400C3EF9548F541EE9547F54075080F200FE3
:103A640003023C97AE4AAF4B7C007D02121EC5D3C5
:103A7400E53F9FEE6480F8E53E6480984024E54687
:103A840020E5067551007550000551AF51EFD394F0
:103A9400504003755150E551C3940A405053080EE9
:103AA400804BAE4AAF4B7C007D02121EC5C3E49F1F
:103AB400FFE49EFEC3E53F9FEE6480F8E53E64802C
:103AC400985024E54620E4067551007550000551D0
:103AD400AF51EFD394504003755150E551C3940A4C
:103AE400400B53080D8006755100755000AE4AAF67
:103AF4004B7C007D02121EC5D3E5419FEE6480F825
:103B0400E5406480984024E54620E706754F00753B
:103B14004900054FAF4FEFD394504003754F50E524
:103B24004FC3940A405D53080B8058AE4AAF4B7C98
:103B3400007D02121EC5C3E49FFFE49EFEC3E5415F
:103B44009FEE6480F8E5406480985031D3E5489452
:103B540000E547648094804024E54620E606754FDE
:103B640000754900054FAF4FEFD394504003754F94
:103B740050E54FC3940A400B5308078006754F0065
:103B8400754900AF3FAE3E126D838E428F43C374BE
:103B9400289543FFE49542FEEF7802C333CE33CE3B
:103BA400D8F9FFAD507C00C3EF9DF545EE9CF5447C
:103BB400C3E544648094805006754400754500E56F
:103BC40051C39450501DAF517E007C007D7F121E66
:103BD400B37C007D50121EC5EF2480FFEF64FFF517
:103BE400FA8027C3E5439428E54264809480501703
:103BF400E550C394A050100550C3E54464809480FC
:103C040040088545FA800375FA00AF41AE40126D55
:103C1400838E428F43C374289543FFE49542FEEF9D
:103C24007802C333CE33CED8F9FFAD497C00C3EF5D
:103C34009DF545EE9CF544C3E544648094805006AC
:103C4400754400754500E54FC39450501DAF4F7E39
:103C5400007C007D7F121EB37C007D50121EC5EFD8
:103C64002480FFEF64FFF5FE803BC3E5439428E521
:103C740042648094805017E549C394A050100549CC
:103C8400C3E54464809480401C8545FE801775FE1E
:103C9400008012755100755000754F00754900750C
:103CA400FA0075FE00E508C454F0FFEF240FF54652
:033CB4008546A0A2
:013CB70022EA
:106D0C004310000043D8000044A2000045110000CD
:106D1C0045B400004622000000C700C70002000A6C
:106D2C000E0F03840E0F038400010001000000000D
:086D3C0000000000000000004F
:106C7200011400011663011200011700011A00C17C
:036C820013C192A9
:0300030002643F55
:10643F00C0E0C083C08263A201C083C082C0D07598
:10644F00D000C006C00720124F20134CD2B330B378
:10645F00020512051AAF1AC3EF64809488401CAF6F
:10646F0017EF3395E0FE74402FF58274003EF583ED
:10647F00E512F07512000517751A00E5122512F5D1
:10648F0012C3E51764809484404F751700D21390A0
:10649F000048E0FF8F12804120123E30133BE5127F
:1064AF002512F512A2D792B3051AAF1AC3EF648063
:1064BF009488401A0517AF17EF3395E0FE74482FF5
:1064CF00F58274003EF583E0FF8F12751A00C3E565
:1064DF0017648094A04002D212D007D006D0D0D03B
:0D64EF0082D08363A201D082D083D0E0323E
:10519200900048E56EF0A3E56FF0E56B2484FFE52F
:1051A2006A3403FE90004AEEF0A3EFF090004CE563
:1051B2004DF0A3E54EF0E5482484FFE5473403FEB5
:1051C20090004EEEF0A3EFF0E50B2484FFE50A34E5
:1051D20003FE900050EEF0A3EFF0900022E0FEA359
:1051E200E0FF900052EEF0A3EFF0900024E0FEA367
:1051F200E0FF900054EEF0A3EFF0900028E0FEA351
:10520200E0FF900056EEF0A3EFF0900058E54AF070
:10521200A3E54BF0300F0B90005AE4F0A37401F0B9
:10522200800890005AE4F0A3E4F0900015E0FFEF4C
:105232003395E0FE90005CEEF0A3EFF0900014E0F6
:10524200FFEF3395E0FE90005EEEF0A3EFF09000EA
:1052520013E0FFEF3395E0FE900060EEF0A3EFF075
:10526200900012E0FFEF3395E0FE900062EEF0A3B3
:10527200EFF0900011E0FFEF3395E0FE900064EE56
:10528200F0A3EFF0900041E0F516900040E4F0A3A7
:105292007463F0C3E516648094884003025377C3B5
:1052A200E516648094805003025377900042E0F543
:1052B20018A3E0F519AF16EF3395E0FEEF25E0FFF6
:1052C200EE33FE74242FF582746D3EF583E493FE73
:1052D200740193FFD3E5199FEE6480F8E5186480AA
:1052E200984021AF16EF3395E0FEEF25E0FFEE3355
:1052F200FE74242FF582746D3EF583E493F51874E1
:105302000193F519AF16EF3395E0FEEF25E0FFEEBE
:1053120033FE74342FF582746D3EF583E493FE748C
:105322000193FFC3E5199FEE6480F8E51864809845
:105332005021AF16EF3395E0FEEF25E0FFEE33FE8E
:1053420074342FF582746D3EF583E493F51874017D
:1053520093F519AF16EF3395E0FEEF25E0FFEE333C
:10536200FE74222FF58274003EF583E518F0A3E562
:1053720019F0125045E516B40805A20FB3920F2298
:03002B0002637DF0
:10637D00C0E0C0F0C083C08263A201C083C082C0F0
:10638D00D075D000C000C001C002C003C004C0055C
:10639D00C006C00775A61E75A6E11509AF09EF70F9
:1063AD006D75090453907790003AE0FEA3E0FFEF7E
:1063BD008EF012209463EA000063EF000163F40095
:1063CD000263F9000363FE00046403000564080022
:1063DD0006640D000764120008000064151267A81A
:1063ED0080261269848021126B44801C1261A68064
:1063FD001712000E8012125C85800D125D9D8008B3
:10640D00125EB1800312571A4390881237D4C2CF4F
:10641D00D007D006D005D004D003D002D001D000D3
:10642D00D0D0D082D08363A201D082D083D0F0D0DF
:02643D00E0324B
:03002300026BD499
:106BD400C0E0C0F0C083C08263A201C083C082C091
:106BE400D075D000C000C001C002C003C004C005FD
:106BF400C006C007C2AC30981AC298E599B43F03E6
:106C0400125382E599B4210B125568D214D215D2CD
:106C140016D217C299D2ACD007D006D005D004D072
:106C240003D002D001D000D0D0D082D08363A2019F
:096C3400D082D083D0F0D0E03210
:03000B000264FC90
:1064FC00C0E0C0F0C083C08263A201C083C082C070
:10650C00D075D000C000C001C002C003C004C005DB
:10651C00C006C007758A00758C4C75A61E75A6E161
:10652C000514AF14C3EF6480948A401630121375AF
:10653C001400751700751A00C213C21275120012DE
:10654C005192E51375F007121E39AFF0EF701B1264
:10655C00413B301804D214D217E57660073018048A
:10656C00D215D21612002E124F961513AF13EF70D0
:10657C000C75134ED218301804D215D216D007D081
:10658C0006D005D004D003D002D001D000D0D0D09A
:0F659C0082D08363A201D082D083D0F0D0E032CE
:10222E00758FFF758921758DFF438780759850D204
:10223E008CD28ED2CA75CB4C75CA0043B81143B737
:10224E0021D28875D90243D84075DA4275DE42C272
:10225E00187513467509017F02125BCF125C1C754F
:10226E007700900040E4F0A37463F020A003126A9C
:10227E001E75A8B275A707125052125074C20F9055
:10228E00006CE0FEA3E0FFEF4E6004D2108002C2AD
:10229E0010900068E0F560A3E0F56190006AE0F54B
:1022AE005AA3E0F55BE57670FC900036E0FCA3E007
:1022BE00FDEC121B807B007A0079207841121A60A7
:1022CE007B007A00793478C31218669001E2E0F848
:1022DE00A3E0F9A3E0FAA3E0FB12195790001E1237
:1022EE002011900038E0FCA3E0FDEC121B807B0077
:1022FE007A0079207841121A607B007A0079B478DE
:10230E00C21218669001E2E0F8A3E0F9A3E0FAA386
:10231E00E0FB12195790001A122011900011E0FCE8
:10232E00EC121B857B007A0079B47844121A60C0D7
:10233E0004C005C006C007900012E0FCEC121B851D
:10234E007B007A0079C07841121A60A804A905AA08
:10235E0006AB07D007D006D005D004121866C0040D
:10236E00C005C006C007900010E0FCEC121B857B78
:10237E00007AC079A87847121A60A804A905AA069F
:10238E00AB07D007D006D005D004121866900044D3
:10239E00122011900014E0FFEF3395E0FEFDFCEFEC
:1023AE002409FFEE3400FEED3400FDEC3400FC7B1E
:1023BE000C7A0079007800126C86A804A905AA068A
:1023CE00AB07900015E0FFEF3395E0FEFDFCEF2428
:1023DE00D0FFEE3407FEED3400FDEC3400FCEB2FA5
:1023EE00FFEA3EFEE93DFDE83CFC7B077A00790002
:1023FE007800121F117B047A0079007800126C8627
:10240E00C004C005C006C007900015E0FFEF33956D
:10241E00E0FEFDFC7B6F7A0179007800121F11D06F
:10242E0003D002D001D000C3EF9BFFEE9AFEED99D0
:10243E00FDEC98FCC004C005C006C007900014E077
:10244E00FFEF3395E0FEFDFC7B137A0179007800F7
:10245E00121F117B097A0079007800126C86A8048D
:10246E00A905AA06AB07D007D006D005D004EB2FDE
:10247E00FBEA3EFAE93DF9E83CF8900013E0FFEF85
:10248E003395E0FEFDFCEB2FFFEA3EFEE93DFDE855
:10249E003CFCEF247AF511EE34E0F510ED3400F546
:1024AE000FEC3400F50E900028E0FEA3E0FFEF6481
:1024BE00014E70487B017A007908C003C002C0014A
:1024CE007B017A0079789001ABEBF0A3EAF0A3E9F7
:1024DE00F0AF11AE10AD0FAC0E9001AE12201190F8
:1024EE000044E0FCA3E0FDA3E0FEA3E0FF9001B2F8
:1024FE00122011D001D002D003124586900028E0A0
:10250E00FEA3E0FFEF4E60030226E17B017A007925
:10251E0008C003C002C0017B017A007978900123C4
:10252E00EBF0A3EAF0A3E9F0AF11AE10AD0FAC0ED5
:10253E00900126122011900044E0FCA3E0FDA3E0E0
:10254E00FEA3E0FF90012A122011D001D002D00389
:10255E00122AB690001AE0FCA3E0FDA3E0FEA3E071
:10256E00FF1259067B547AE379457840121957C009
:10257E0004C005C006C007900016E0FCA3E0FDA352
:10258E00E0FEA3E0FF12591CA804A905AA06AB079A
:10259E00D007D006D005D004121957C004C005C00C
:1025AE0006C007900078E0FCA3E0FDA3E0FEA3E0E8
:1025BE00FF125906A804A905AA06AB07D007D00634
:1025CE00D005D004121957C004C005C006C007AF0D
:1025DE0011AE10AD0FAC0EC004C005C006C0077F13
:1025EE00AB7EAA7D2A7C3C900044E0F8A3E0F9A3E0
:1025FE00E0FAA3E0FB12186690015E122011D007DC
:10260E00D006D005D004120D30C004C005C006C0DF
:10261E0007AF11AE10AD0FAC0EC004C005C006C0A2
:10262E00077FAB7EAA7D2A7CBC900044E0F8A3E035
:10263E00F9A3E0FAA3E0FB12186690015E122011D6
:10264E00D007D006D005D004120D30D003D002D062
:10265E0001D0001218627B007A0079877843121A33
:10266E0060A804A905AA06AB07D007D006D005D0EE
:10267E00041218667B007A00797A78441219571280
:10268E001BB98E0C8F0DAC0CAD0DEC121B80C00463
:10269E00C005C006C00790003CE0FEA3E0FFEF7847
:1026AE0002C333CE33CED8F9FF740C2FF582746D7E
:1026BE003EF583121FE1D007D006D005D0041219C3
:1026CE00577B007A00797A7844121A60121BB98E01
:1026DE001B8F1C900028E0FEA3E0FFEF64024E70FB
:1026EE001490007812201D3F82D0E5900008122031
:1026FE001D40C39DB2900028E0FEA3E0FFEF6403EF
:10270E004E701490007812201D3F3566CF90000851
:10271E0012201D40A73B64900028E0FEA3E0FFEFCF
:10272E0064044E701490007812201DBF018FC59066
:10273E00000812201D40953F7D900028E0FEA3E08A
:10274E00FFEF64054E701490007812201D3EC44DAC
:10275E000190000812201D3FB91687900028E0FE58
:10276E00A3E0FFEF64064E701490007812201D3F18
:10277E0032B6AE90000812201D401F2B029000288A
:10278E00E0FEA3E0FFEF64074E7014900078122075
:10279E001D0000000090000812201D40BC7AE19040
:1027AE000028E0FEA3E0FFEF64084E706790003251
:1027BE00E0FCA3E0FDEC121B807B007A0079207810
:1027CE0041121A609001E2E0F8A3E0F9A3E0FAA347
:1027DE00E0FB121957900008122011900034E0FC13
:1027EE00A3E0FDEC121B807B007A00792078411269
:1027FE001A607B007A0079B478C21218669001E2F2
:10280E00E0F8A3E0F9A3E0FAA3E0FB121957900059
:10281E0078122011900028E0FEA3E0FFC3EF940988
:10282E00EE648094804003022935900044E0FCA3BE
:10283E00E0FDA3E0FEA3E0FFC004C005C006C00794
:10284E00AF11AE10AD0FAC0E9001CE122011D0070D
:10285E00D006D005D00412494E9001881220117B6B
:10286E00017A00790CC003C002C0017B017A0079A5
:10287E0000900185EBF0A3EAF0A3E9F0900008E0E8
:10288E00FCA3E0FDA3E0FEA3E0FF90018C1220115B
:10289E00900078E0FCA3E0FDA3E0FEA3E0FF900132
:1028AE0090122011D001D002D0031232BD90002818
:1028BE00E0FEA3E0FFEF4E705A900000E0FCA3E0B4
:1028CE00FDA3E0FEA3E0FF1259067B007A5079C704
:1028DE007845121957C004C005C006C0079000E81D
:1028EE0012201D48B98C00D007D006D005D0041296
:1028FE0068E7A804A905AA06AB07900000E0FCA3B0
:10290E00E0FDA3E0FEA3E0FF121862900004122087
:10291E00118014900000E0FCA3E0FDA3E0FEA3E014
:10292E00FF900004122011900028E0FEA3E0FFEFBC
:10293E0064094E705C90002EE0FCA3E0FDEC121BCF
:10294E00807B007A0079207841121A609001E2E0D3
:10295E00F8A3E0F9A3E0FAA3E0FB12195790000CDC
:10296E00122011900030E0FCA3E0FDEC121B807BE6
:10297E00007A0079207841121A609001E2E0F8A303
:10298E00E0F9A3E0FAA3E0FB12195790000412201D
:10299E0011900028E0FEA3E0FFEF640A4E705C90F9
:1029AE00002AE0FCA3E0FDEC121B807B007A00798C
:1029BE00207841121A609001E2E0F8A3E0F9A3E05A
:1029CE00FAA3E0FB12195790000C12201190002C64
:1029DE00E0FCA3E0FDEC121B807B007A00792078EE
:1029EE0041121A609001E2E0F8A3E0F9A3E0FAA325
:1029FE00E0FB1219579000041220119001E2E0F84A
:102A0E00A3E0F9A3E0FAA3E0FB90000CE0FCA3E046
:102A1E00FDA3E0FEA3E0FF121A607BCD7ACC794CC9
:102A2E00783D1218667B007A00792078411219578A
:102A3E00121BB98E6E8F6F9001E2E0F8A3E0F9A33E
:102A4E00E0FAA3E0FB900004E0FCA3E0FDA3E0FEAF
:102A5E00A3E0FF121A607BCD7ACC794C783D121828
:102A6E00667B007A0079207841121957121BB98EB5
:102A7E006A8F6B7F007E007D207C41900078E0F8AD
:102A8E00A3E0F9A3E0FAA3E0FB1219579001E2E0EC
:102A9E00F8A3E0F9A3E0FAA3E0FB121A60121BB947
:082AAE008E0A8F0B0222B322F5
:105B6800EFC0E0C283740F125B9D7430125BA774A0
:105B780005125B9D7430125BA77401125B9D743033
:105B8800125BA77401125B9DD0E014600274084494
:105B980020125BB5227D000000DDFCD5E0F7225421
:105BA800F053800F4280C282D283C28322C2828095
:105BB80002D282C0E0125BC3D0E0C454F053800F1D
:105BC8004280D283C28322125B68125C017406127F
:105BD8005BB5125C01740E125BB5125C01740112A4
:105BE8005BB5125C017440125BB5125C4E125C012D
:105BF8007480125BB5125C2E22740A125B9D22EF30
:105C0800C0E0125C01D0E0125BB922125C017402A0
:105C1800125BB522125C017401125BB522125C01A1
:105C2800740E125BB522125C01740C125BB5221261
:105C38005C01740F125BB522EFC0E0125C01D0E08A
:105C48004480125BB522905C5D7E28E493FF125C71
:105C580007A3DEF7220004040E0E1F1F00001F1FFB
:105C68000E0E04040000101C1F1C10000000010789
:0D5C78001F070100000E11171917110E0073
:106D6B007A107B00EE6BFB8BF053F080ABF033EFC4
:086D7B0033FFEE33FEDAEE22D5
:106AB300900203EEF0A3EFF0900203E0FEA3E0FFE9
:106AC3007C037DE8121EC5EF2430F5993099FDC291
:106AD30099900203E0FEA3E0FF7C037DE8121EC54C
:106AE3007E007F64CFCDCFCECCCE121EC5EF243037
:106AF300F5993099FDC299900203E0FEA3E0FF7C73
:106B0300007D64121EC57E007F0ACFCDCFCECCCED2
:106B1300121EC5EF2430F5993099FDC299900203F6
:106B2300E0FEA3E0FF7C007D0A121EC5AF05EF2443
:106B330030F5993099FDC2997599003099FDC29944
:016B4300222F
:105382009001F912201D000186A020983E9001F99B
:10539200E0FCA3E0FDA3E0FEA3E0FFEC4D4E4F6076
:1053A2002A9001F9E0FCA3E0FDA3E0FEA3E0FF7B6D
:1053B200FF7AFF79FF78FFEF2BFFEE3AFEED39FD22
:1053C200EC38FC9001F912201180BFC298AF99EF1E
:1053D20012206E542761543362543F63544764541D
:1053E2005365545F66546B67547768548369548F6E
:1053F2006A549B6B54A76C54B36D54BF6E54CD6FFB
:1054020054D57054E37154EB7254F97355017455C9
:105412001475552276553077553E78554C79555A44
:105422007A00005567900022E0FEA3E0FF126AB303
:1054320022900024E0FEA3E0FF126AB322AF4BAE3B
:105442004A126AB322900028E0FEA3E0FF126AB378
:105452002290002AE0FEA3E0FF126AB32290002C01
:10546200E0FEA3E0FF126AB32290002EE0FEA3E06A
:10547200FF126AB322900030E0FEA3E0FF126AB38B
:1054820022900032E0FEA3E0FF126AB322900034C1
:10549200E0FEA3E0FF126AB322900036E0FEA3E032
:1054A200FF126AB322900038E0FEA3E0FF126AB353
:1054B2002290003AE0FEA3E0FF126AB322E50D2437
:1054C20088FFE50C3413FE126AB322AF4EAE4D12C2
:1054D2006AB322E5482484FFE5473403FE126AB327
:1054E20022AF6FAE6E126AB322E56B2484FFE56AC7
:1054F2003403FE126AB322AF0BAE0A126AB3223031
:105502000F087F017E00126AB3227F007E00126ABA
:10551200B322900010E0FFEF3395E0FE126AB3224F
:10552200900011E0FFEF3395E0FE126AB322900083
:1055320012E0FFEF3395E0FE126AB322900013E00F
:10554200FFEF3395E0FE126AB322900014E0FFEF02
:105552003395E0FE126AB322900015E0FFEF339517
:05556200E0FE126AB337
:015567002221
:106703009001EEE4F0A3E4F09001F4E4F09001F4DE
:10671300E0FFD3EF64809483400302679F9001F00E
:1067230012201D000186A020983E9001F0E0FCA3FA
:10673300E0FDA3E0FEA3E0FFEC4D4E4F602A900185
:10674300F0E0FCA3E0FDA3E0FEA3E0FF7BFF7AFF04
:1067530079FF78FFEF2BFFEE3AFEED39FDEC38FCC5
:106763009001F012201180BFC2989001EEE0FEA3C9
:10677300E0FF7C007D0A121EB3AD997C00EF2DFF74
:10678300EE3CFEEF24D0FFEE34FFFE9001EEEEF080
:10679300A3EFF09001F4E004F00267109001EEE043
:0467A300FEA3E0FF72
:0167A70022CF
:105568009001FD12201D000186A020983E9001FDAB
:10557800E0FCA3E0FDA3E0FEA3E0FFEC4D4E4F608E
:105588002A9001FDE0FCA3E0FDA3E0FEA3E0FF7B81
:10559800FF7AFF79FF78FFEF2BFFEE3AFEED39FD3A
:1055A800EC38FC9001FD12201180BFC298AF99EF32
:1055B80012206E560161561062561F63562E6456AD
:1055C8003D65564C66565B67566A685679695688D3
:1055D8006A56976B56A66C56B56D56C47256C97303
:1055E80056CC7456D27556DE7656EA7756F6785704
:1055F8000279570E7A00005719126703900022EEBD
:10560800F0A3EFF012504522126703900024EEF049
:10561800A3EFF012504522126703900026EEF0A384
:10562800EFF012504522126703900028EEF0A3EF26
:10563800F01250452212670390002AEEF0A3EFF013
:105648001250452212670390002CEEF0A3EFF012DF
:1056580050452212670390002EEEF0A3EFF012508F
:105668004522126703900030EEF0A3EFF012504588
:1056780022126703900032EEF0A3EFF01250452299
:10568800126703900034EEF0A3EFF0125045221297
:105698006703900036EEF0A3EFF012504522126730
:1056A80003900038EEF0A3EFF01250452212670382
:1056B80090003AEEF0A3EFF012504522D20DD2112D
:1056C80022D21122A20FB3920F2212670390001068
:1056D800EFF0124F4122126703900011EFF0124FC2
:1056E8004122126703900012EFF0124F4122126715
:1056F80003900013EFF0124F412212670390001439
:10570800EFF0124F4122126703900015EFF0124F8D
:01571800414F
:01571900226D
:10185F00021C25E86480F8E933E83360110460F076
:10186F00ED33EC337009E8FCE9FDEAFEEBFF2204EF
:10187F0060DED3EB9FEA9EE99DE8C2E78CF0C2F7EA
:10188F0095F0400CE8CCF8E9CDF9EACEFAEBCFFBB6
:10189F00121BF085D0F05804700320D5B3E8047004
:1018AF00075002B2D5021C2F92D5EC0460F7E4CC9E
:1018BF00C0E0C398F8603B94186008400DD0E0FB7F
:1018CF00021C07E4FBFAC9FC8028E830E406E4C9EF
:1018DF00FBE4CAFCE830E305E4C9CACBFCE85407D3
:1018EF006010F8C3E913F9EA13FAEB13FBEC13FCDE
:1018FF00D8F130F52FC3E49CFCEF9BFFEE9AFEED81
:10190F0099FDD0E0FBEF4E4D4C701222DB03021C11
:10191F002CEC2CFCEF33FFEE33FEED33FDED30E717
:10192F00EB021C07EF2BFFEE3AFEED39FDD0E0FB8B
:10193F0050130BBB0003021C2FED13FDEE13FEEF34
:08194F0013FFEC13FC021C075E
:10195700EC4D6011E8497017ED33EC3304600DE48A
:10196700FCFFFEFD22E933E8330470F8021C251260
:101977001BF058046009E4CC248150062850090262
:101987001C2F284003021C2CC0E0EB4A7044B9808E
:1019970006D0E0FB021C1BEF4E701CBD8008EBFF5E
:1019A700EAFEE9FD80EBE98DF0A4FEE5F0021A40BE
:1019B700E9CDF9EAFEEBFFEF89F0A4FCE5F0CE896B
:1019C700F0A42EFFE435F0CD89F0A42DFEE435F028
:1019D7008067EF4E7005BD80D780C3EF8BF0A4AC56
:1019E700F0EE8BF0A42CFCE435F0F8EF8AF0A42C91
:1019F700E5F038FCE433CB8DF0A42CFCE5F03BF8A4
:101A0700EE8AF0A42CFCE5F038F8E433CF89F0A493
:101A17002CFCE5F038CF3400CE89F0A42FFFE5F099
:101A27003EFEE433C98DF0A42EFEE5F039CD8AF0F1
:101A3700A42FFFE5F03EFEE43DFD33D0E0FB500769
:101A47000BBB000F021C2FEC2CFCEF33FFEE33FE19
:061A5700ED33FD021C0747
:101A5D00021C2FEC5D046005E859047003021C257F
:101A6D00121BF0580460F6EC4860F2EC7004FDFEB9
:101A7D00FF22C860DB2481C85009C398600250065C
:101A8D00021C2C9850CAF582E9294B4A7005AB828D
:101A9D00021C1B75F0007C1A7880C3EF9BEE9AED4B
:101AAD0099400DC3EF9BFFEE9AFEED99FDE842F0D4
:101ABD00DC23ACF0D0E0FFD0E0FED0E0FDAB822027
:101ACD00E7101BEB60BAEC2CFCEF33FFEE33FEEDB1
:101ADD0033FD021C07E803F830E705C0F075F00090
:101AED00EF2FFFEE33FEED33FD40B830E7C280AA95
:101AFD0074F8CC6480CCC86480C8F582046043C39C
:101B0D00EB9FF5F0EA9E42F0E99D42F0E89C45F02E
:101B1D0060305018E5825FFFE582F42B5582FB5053
:101B2D00210ABA001D09B90019088016E5825BFB70
:101B3D00E582F42F5582FF50090EBE00050DBD0044
:101B4D00010CC3EB9FF5F0EA9E42F0E99D42F0E8EF
:0D1B5D009C45F06007CC4820E701B3EC2266
:101B6A00ED33EC33600A047003BD8004ECB2E7FC89
:011B7A002248
:101B7B0075F020800E75F010800575F0087D007EE5
:101B8B00007F003392D530D503121F60EC33401029
:101B9B00EF33FFEE33FEED33FDEC33FCD5F0ED22EE
:0E1BAB00E5F0247EA2D513CC92E7CDCEFF222A
:101BB900EDD2E7CD33EC3392D524814006E4FFFE24
:101BC900FDFC22FCE4CFCECDCC24E0501174FF8083
:101BD900EDC3CC13CCCD13CDCE13CECF13CF047020
:071BE900F030D5DE021F60A1
:103CB800E57B24F3F582E43400F583E0057B22906C
:103CC80000F03009039000F3E475F00112204E0271
:103CD8001E5B2002E97F2ED2028018EF540F249039
:103CE800D43440D4FF30060BEF24BFB41A0050037D
:103CF8002461FFE57C6002157C057FE57F70020585
:103D08007E30090E9000F0E475F00112204EEF02AB
:103D18001EA1026D447403D2098003E4C209F57B35
:103D28009000F0122065E4F57CF57EF57FE57C6077
:103D3800077F20123CFB80F5757DFFC203C202C2DB
:103D480004C205C207C208C20A123CC7FF700D3080
:103D580009057F00123D0CAF7FAE7E22B4255FC2FD
:103D6800D5C206123CC7FF24D0B40A00501A75F019
:103D78000A787C30D50508B6FF0106C6A426F620C9
:103D8800D5047002D20580D924CFB41A00EF5004AC
:103D9800C2E5D206023FFED20380C6D20280C0D25C
:103DA8000480BCD2D580BAD20780B47F20123CFBF5
:103DB8002004077401B57C0040F1123CB8FF123CA6
:103DC800FB023D35D20AD2088095123CB8FB123C62
:103DD800B8FA123CB8F94A4B700679FC7A407BFF76
:103DE80020042EE57C602A7E008E82758300121ED8
:103DF8007460060EEE657D70F0C2D5EBC0E0EAC0D7
:103E0800E0E9C0E0EE12405FD0E0F9D0E0FAD0E09F
:103E1800FB121E5BFF60AAEBC0E0EAC0E0E9C0E06D
:103E2800123CFBD0E02401F9D0E03400FAD0E0FBEA
:103E3800E57D0460DCD57DD98087D20480A212405C
:103E48004160F7E57D700104121C3AA97D600DE51B
:103E58007D600914F57D1240E9EF60F3EA30E7026E
:103E6800F404C3995079EAF4257D0430E701E404A9
:103E7800F57D800D12404160C1EA057D257D121C4B
:103E88003AEA90011FF030E701E4257D04D57D046E
:103E98002007011412405FE4C0E01240E990011FBE
:103EA800E0601320E70714F0123CE3802204F0D00E
:103EB800E014C0E07F00123CE3E57D6007123CDAC5
:103EC800157D800B300703123CDAD0E0023D35D077
:103ED800E00480C4124041609EE57D04121C3A90C3
:103EE800011FEAF0E57D2007026001042404124066
:013EF8005F6A
:103EF90074FF04C0E01240E9123CE3E57D200702AB
:103F09006003123CDAD0E0B57DE87F45123CED90C4
:103F1900011FE07F2B30E7047F2DF404C0E0123C41
:103F2900FBD0E075F00A84C0F0123CE4D0E0123C0A
:103F3900E4023D35791080027908C208C20A800876
:103F4900D2D5790A8004790AC2D5E57D047002F5D3
:103F59007DE4FAFDFEFF123CB8FC7B082003131236
:103F69003CB8FD7B1030020A123CB8FE123CB8FF87
:103F79007B20EC3382D592D55013C3E43002069FDF
:103F8900FFE49EFEE42003039DFDE49CFCE4CBF8E2
:103F9900C203EC700CCFCECDCCE824F8F870F380D6
:103FA90017C3EF33FFEE33FEED33FDEC33FCEB3398
:103FB900FB994002FB0FD8E9EB300305F8D0E0C4C8
:103FC90048B203C0E00AEC4D4E4F78207B0070C226
:103FD900EAB57D0040BCC0E0124061D0F0D0E020DD
:103FE9000304C4C0E0C4B203C0F0123CE4D0F0D56D
:103FF900F0EB023D3512206E3DD2533F3D583DA3B3
:104009004C3D9F423F414F3F49443F49493DB84399
:104019003F4F553E7C463EDC453E4647411C503DA0
:10402900A72D3DAB2E3DCE2B3DAF233DCC204105E9
:104039002A3D674800003DC6E57DB4FF03757D064E
:10404900123CB8FC123CB8FD123CB8FE123CB8FF59
:10405900900118021C77790AA2D5200514300709A6
:10406900B910020404B9080104A2D52008025001BC
:10407900042004689204B57C005034C0E07F2030ED
:1040890005197F30A20472087207500F1240B8C296
:1040990004C208C207C20A7F30800F300703E9C093
:1040A900E0123CFB300703D0E0F9D0E0B57CCC301E
:1040B90007177F30B9100C123CFB7F583006077F79
:1040C900788003B90803123CFB3004057F2D023CBC
:1040D900FB7F20200AF87F2B2008F322920480CF4F
:1040E9007F00B40700500B2418F582E43401F583EE
:1040F900E0FF22286E756C6C2900D203123CB8309F
:1041090003F8C203787C30D50108F6023D672D50CB
:10411900434958123CB82403B405004001E49041D6
:104129001793123CEC743A123CECD205757C0402EC
:024139003F3D08
:0D6DEA00ED33EC3360065004EC6480FC22B5
:10665700021C2522EDA2E7D2E7F9EC3340F260F302
:10666700B4FF08ED547F70E8021C2FF82481C2E0C4
:10667700C0E0F40428FAC313FCED92E7FD9000E4B0
:10668700122011EEA2E7E9BA7F02C3133400940087
:10669700FA75F091A4E5F013F494FE8AF0A433E5BB
:1066A700F033248CD313FDE492E7FE7F007C3F7523
:1066B7008302ECC0E0F8EDC0E0F9EEC0E0FAEFC00D
:1066C700E0FB8583F09000E4121FB985F083121A6E
:1066D70060D0E0FBD0E0FAD0E0F9D0E0F81218661D
:1066E700ED6480FD30E7011CD583C7ED33CC33F86B
:0C66F700D0E0A2E71328C313CC13FD224F
:1068E7009000E41220119000E8E0F8A3E0F9A3E09B
:1068F700FAA3E0FB9000E4E0FCA3E0FDA3E0FEA325
:10690700E0FF121A60125A669000E41220119000FC
:10691700E8E030E7599000E4E0FCA3E0FDA3E0FEE7
:10692700A3E0FFECC0E0EDC0E0EEC0E0EFC0E0E4C4
:10693700FFFEFDFC9000E4E0F8A3E0F9A3E0FAA372
:10694700E0FB121AFD7BDB600250087A0F79497869
:106957004080067A0F794978C0D0E0FFD0E0FED0BA
:10696700E0FDD0E0FC1218669000E41220119000C0
:0D697700E4E0FCA3E0FDA3E0FEA3E0FF22AE
:1058BE003A70FA83BCAAE9E43E81E0F8BF9DE9E6BE
:1058CE003F80000039283C1ABB9969663DA335E339
:1058DE00BF255DE73FC90FDB418DDBCCC44936EEFA
:1058EE0045C9913FC5B0F83D3F800000C317F53460
:1058FE00452FFA73C60AFDDD1259C704A2E19200C4
:10590E001420E0159058BE7404121D7C803012597C
:10591E00C730E102B20020E0EBA883A9829000E438
:10592E00122011898288839058D27404121D7C85AE
:10593E0082F09000E4121FD585F082121957ED4CBB
:10594E006007300004EC6480FC221259C7C0E0A846
:10595E0083A9829000E4122011898288839058F6E0
:10596E007403121D7C8582F09000E4121FD585F021
:10597E00821219579000E4E0CCF0A3E0CDF0A3E042
:10598E00CEF0A3E0CFF09058E67403121D7CD082C7
:10599E008582F09000E4121FD585F082E58230E01A
:1059AE0007121A60B2008096EFCBFFEECAFEEDC969
:1059BE00FDECC8FC121A608085ED33EC547FCC33BD
:1059CE00920024605007D0E0D0E0021C257B837A41
:1059DE00F97922783E121957EDF933ECF833248118
:1059EE005011EFFBEEFA121BB9121B7BECB2E7FC67
:1059FE00121866ED33EC33602F2403F8C313FCED5D
:105A0E0092E7FDE82481E4501FECF8EDF9EEFAEF91
:105A1E00FB121BB9EF04C2E0FCF582121B85ECB23F
:105A2E00E7FC121866E58203FAED33EC33600714D7
:085A3E0013FCED92E7FDEA22E2
:105A4600BE1249253E4CCCCDBEAAAAAB3F80000073
:105A56003E7ADBB03EED63383F24BC7D3F490FDB29
:105A6600ED33ECC2E7CC339200B4FF13ED547F6004
:105A760003021C257FDB7E0F7DC97C3F025B5BC278
:105A860001C3947F401E7007EDD2E794904015EF56
:105A9600FBEEFAEDF9ECF87F007E007D807C3F128C
:105AA6001A60D201ED33EC33248430E705E4C0E01C
:105AB600806B04FAEDD2E754F0C333DAFD540734B1
:105AC600002323C0E0CCC0E0F8EDC0E0F9EEC0E072
:105AD600FAEFC0E0FBE4121B85EC24FEFC9000EC20
:105AE6001220111219577B007A007980783F12181C
:105AF600669000ECE0B2E7CCF0A3E0CDF0A3E0CEF8
:105B0600F0A3E0CFF0D0E0FBD0E0FAD0E0F9D0E0AF
:105B1600F81218669000EC121FD5121A609000EC6D
:105B2600122011905A467403121D7C9000EC121F2D
:105B3600D5121957D0E0600F2452F582E4345AF595
:105B460083121FE112186630010B7BDB7A0F79C9CD
:105B560078BF121866ED33EC336006ECA20092E7CC
:025B6600FC221F
:1060B6009000E412201174FFFFFEFDFC9000E4E066
:1060C600F8A3E0F9A3E0FAA3E0FBC3121F6E603861
:1060D6007F807E967D187C4B9000E4E0F8A3E0F983
:1060E600A3E0FAA3E0FB121AFD6002501B7F807E3C
:1060F600967D187CCB9000E4E0F8A3E0F9A3E0FAE3
:10610600A3E0FB121AFD500F9000E4E0FCA3E0FDB3
:10611600A3E0FEA3E0FF229000E4E0FCA3E0FDA3E1
:10612600E0FEA3E0FF121BB99000E81220119000D8
:10613600E8E0FCA3E0FDA3E0FEA3E0FFEC121B7B7E
:10614600C8ECC8C9EDC9CAEECACBEFCB9000E4E0F3
:10615600FCA3E0FDA3E0FEA3E0FF121862E4FBFA55
:10616600F9F8121AFD602640249000E8E0FCA3E04E
:10617600FDA3E0FEA3E0FFEF24FFFFEE34FFFEEDFC
:1061860034FFFDEC34FFFC9000E81220119000E88B
:10619600E0FCA3E0FDA3E0FEA3E0FFEC121B7B22E4
:101BF000E9D2E7C933E833F892D5EDD2E7CD33EC3B
:071C000033FC5002B2D522B3
:101C0700EC30E7100FBF000C0EBE00080DBD00043E
:101C17000BEB6014A2D5EB13FCED92E7FD2274FFEA
:101C2700FCFDFEFF22E480F8A2D574FF13FC7D8043
:031C3700E480EF57
:101C3A00F920E73624F950037907E4F42402FBE596
:101C4A0082158270021583DBF6E024FB501BE960E3
:101C5A0014E4F0E582158270021583E004F0B40AF8
:0D1C6A0008E4F0D9EE7401F00A22C2D52280
:101C7700ED33EC3392D5FA602AB4FF33EDC2E77B3C
:101C8700FF60067A1C799CE4227A1C79A520D5048A
:101C97007A1C79A0224E614E002B494E46002D49F1
:101CA7004E4600E47A08F0A3DAFC7B00740722C0F2
:101CB70083C082ECC0E0EDC0E0EEC0E0EFC0E0EA38
:101CC70075F010A4CAABF075F04DA42BFBE435F00A
:101CD700FCEA2410FAEB34C5FBEC34D9FCEDC2E77F
:101CE700FF75F056A4F42411C5F0F434C58FF0A4A1
:101CF7002AE5F03BE43CF020E714121DF9D0E0FFA1
:101D0700D0E0FED0E0FDD0E0FC121A608014F404AD
:101D1700121DF9D0E0FFD0E0FED0E0FDD0E0FC12CC
:101D27001957D082D083E0FAEDD2E7CD33EC3324D4
:101D370082FBE4C3CF33CFCE33CECD33CD33DBF30A
:101D47007B0775F00A846004F0A31B0AE5F0F0A393
:101D57008FF0740AA4FFACF08EF0740AA42CFEACCA
:101D6700F050010C8DF0740AA42CFDE435F0F0A3BB
:051D7700DBDE74072211
:101D7C00C0E0EFFBEEFAEDF9ECF8121957D0E0F5F4
:101D8C00F0EFFBEEFAEDF9ECF8121FC5A3A3A3A339
:101D9C00E8C0E0E9C0E0EAC0E0EBC0E0C0F0121936
:101DAC0057121FE1A3A3A3A3121866D0F0D0E0FB37
:0D1DBC00D0E0FAD0E0F9D0E0F8D5F0D42264
:101DC9003F8000004120000042C80000447A000022
:101DD900461C400047C35000497424004B189680A4
:101DE9004CBEBC205A0E1BCA6753C21C749DC5AE9B
:101DF900FB60065407601C2323121E27EB5438602E
:101E090009121E13121E22121957ECF8EDF9EEFAF7
:101E1900EFCB22EB121E2280F1543803241C901DB3
:101E2900C9FE93FC0EEE93FD0EEE930ECE93FF22A8
:1068670002222EE493A3F8E493A34003F68001F2F7
:1068770008DFF48029E493A3F85407240CC8C33332
:10688700C4540F4420C8834004F456800146F6DF01
:10689700E4800B0102040810204080906C3DE47EE8
:1068A700019360BCA3FF543F30E509541FFEE493F6
:1068B700A360010ECF54C025E060A840B8E493A3BD
:1068C700FAE493A3F8E493A3C8C582C8CAC583CAE8
:1068D700F0A3C8C582C8CAC583CADFE9DEE780BEA0
:016C8500000E
:101E3900C2D530F707B2D563F0FF05F030E70CB231
:101E4900D5F4048463F0FF05F080018430D502F4F1
:021E5900042261
:101E5B00BB010689828A83E0225002E722BBFE0285
:091E6B00E32289828A83E49322B8
:101E7400BB010CE58229F582E5833AF583E0225023
:101E840006E92582F8E622BBFE06E92582F8E2226D
:0D1E9400E58229F582E5833AF583E4932287
:101EA100BB010689828A83F0225002F722BBFE0120
:021EB100F3221A
:101EB300EF8DF0A4A8F0CF8CF0A428CE8DF0A42E43
:021EC300FE22FD
:101EC500C2D5EC30E709B2D5E4C39DFDE49CFCEE38
:101ED50030E715B2D5E4C39FFFE49EFE1220C1C3CF
:101EE500E49DFDE49CFC80031220C130D507C3E4CA
:061EF5009FFFE49EFE22A7
:101EFB00C5F0F8A3E028F0C5F0F8E5821582700272
:061F0B001583E038F0220E
:101F1100E88FF0A4CC8BF0A42CFCE98EF0A42CFC6F
:101F21008AF0EDA42CFCEA8EF0A4CDA8F08BF0A4ED
:101F31002DCC3825F0FDE98FF0A42CCD35F0FCEB4C
:101F41008EF0A4FEA9F0EB8FF0A4CFC5F02ECD3911
:0F1F5100FEE43CFCEAA42DCE35F0FDE43CFC227E
:106C8600C2D5E830E70FB2D5E4C39BFBE49AFAE439
:106C960099F9E498F8EC30E717B2D5126CBC1221DA
:106CA60052E4C39BFBE49AFAE499F9E498F880036A
:106CB60012215230D50DE4C39FFFE49EFEE49DFDF4
:046CC600E49CFC222C
:0E1F6000C3E49FFFE49EFEE49DFDE49CFC2292
:101F6E00EB9FF5F0EA9E42F0E99D42F0E89C45F0C9
:011F7E002240
:101F7F00BB010789828A83021FB95005E9F8022144
:101F8F00E4BBFE05E9F80221F089828A83021FC5AE
:101F9F00BB010789828A830220115005E9F80222CA
:0A1FAF0016BBFE05E9F8022222220B
:0C1FB900E0FCA3E0FDA3E0FEA3E0FF229B
:101FC500E493FC740193FD740293FE740393FF2262
:0C1FD500E0F8A3E0F9A3E0FAA3E0FB228F
:101FE100E493F8740193F9740293FA740393FB2256
:101FF100BB010789828A83021FD55005E9F80221B6
:10200100FCBBFE05E9F802220989828A83021FE1ED
:0C201100ECF0A3EDF0A3EEF0A3EFF02242
:10201D00A8828583F0D083D082122034122034120E
:10202D002034122034E473E493A3C583C5F0C58333
:10203D00C8C582C8F0A3C583C5F0C583C8C582C80D
:01204D002270
:10204E00F8E0FBA3A3E0F925F0F0E582158270021B
:07205E001583E0FA38F022BF
:09206500EBF0A3EAF0A3E9F0227C
:10206E00D083D082F8E4937012740193700DA3A301
:10207E0093F8740193F5828883E473740293686015
:06208E00EFA3A3A380DF15
:10209400D083D082F8E4937012740193700DA3A3DB
:1020A40093F8740193F5828883E473740293B5F012
:0D20B400067403936860E9A3A3A3A380D87A
:106D4400EFB40A07740D126D4F740A309811A899A4
:106D5400B8130CC2983098FDA899C298B811F630AF
:076D640099FDC299F5992287
:106D8300C3EE6480948040028007C3E49FFFE49EC7
:026D9300FE22DE
:1020C100BC000BBE0029EF8DF084FFADF022E4CC03
:1020D100F875F008EF2FFFEE33FEEC33FCEE9DECCC
:1020E100984005FCEE9DFE0FD5F0E9E4CEFD22ED12
:1020F100F8F5F0EE8420D21CFEADF075F008EF2F5C
:10210100FFED33FD4007985006D5F0F222C398FD4C
:052111000FD5F0EA22E9
:1021160075F008758200EF2FFFEE33FECD33CDCC80
:1021260033CCC58233C5829BED9AEC99E582984003
:102136000CF582EE9BFEED9AFDEC99FC0FD5F0D6E0
:10214600E4CEFBE4CDFAE4CCF9A88222B800C1B90A
:102156000059BA002DEC8BF084CFCECDFCE5F0CB48
:10216600F97818EF2FFFEE33FEED33FDEC33FCEB81
:1021760033FB10D703994004EB99FB0FD8E5E4F93C
:10218600FA227818EF2FFFEE33FEED33FDEC33FC29
:10219600C933C910D7059BE99A4007EC9BFCE99A1D
:1021A600F90FD8E0E4C9FAE4CCFB2275F010EF2F62
:1021B600FFEE33FEED33FDCC33CCC833C810D70762
:1021C6009BEC9AE899400AED9BFDEC9AFCE899F89D
:0E21D6000FD5F0DAE4CDFBE4CCFAE4C8F92230
:0C21E400E6FC08E6FD08E6FE08E6FF2227
:0C21F000E2FC08E2FD08E2FE08E2FF222B
:0D21FC00E6FB08E6F908E6FA08E6CBF82253
:0D220900E2FB08E2F908E2FA08E2CBF82255
:0C221600ECF608EDF608EEF608EFF622F4
:0C222200ECF208EDF208EEF208EFF222F8
:00000001FF
